 eboot

 Timestamp is 4da293db (Mon Apr 11 17:38:35 2011)

 Preferred load address is 00010000

 Start         Length     Name                   Class
 0001:00000000 000002f8H .astart                 CODE
 0001:00000300 000050afH .rdata                  CODE
 0001:000053b0 00000022H .rdata$debug            CODE
 0001:000053e0 0001b348H .text                   CODE
 0001:00020728 000000a8H .xdata                  CODE
 0001:000207d0 00000000H .edata                  CODE
 0002:00000000 00005a0cH .data                   DATA
 0002:00005a20 0001efacH .bss                    DATA
 0003:00000000 00000e20H .pdata                  DATA

  Address         Publics by Value              Rva+Base       Lib:Object

 0000:00000000       ___safe_se_handler_table   00000000     <absolute>
 0000:00000000       ___safe_se_handler_count   00000000     <absolute>
 0001:00000000       StartUp                    00011000 f   bootcmn:startup.obj
 0001:000000f4       g_oalAddressTable          000110f4     bootcmn:startup.obj
 0001:0000016c       KernelStart                0001116c f   bootcmn:startup.obj
 0001:00000260       Launch                     00011260 f   bootcmn:startup.obj
 0001:0000031c       ??_C@_08PLDKGPEJ@17?335?359?$AA@ 0001131c     eboot.obj
 0001:00000328       ??_C@_0M@CJGCCEJL@Apr?511?52011?$AA@ 00011328     eboot.obj
 0001:00000338       ??_C@_0EK@BLGPAFDM@Microsoft?5Windows?5CE?5Ethernet?5Bo@ 00011338     eboot.obj
 0001:00000384       ??_C@_05DFLKGENG@Topaz?$AA@ 00011384     eboot.obj
 0001:0000038c       ??_C@_0DO@GKLPKMK@ERROR?3?5Failed?5to?5detect?5and?5init@ 0001138c     eboot.obj
 0001:000003cc       ??_C@_0CJ@HMMHCENL@ERROR?3?5EbootWaitForHostConnect?5f@ 000113cc     eboot.obj
 0001:000003f8       ??_C@_0FA@OIIAKJBG@INFO?3?5EbootWaitForHostConnect?5?$CII@ 000113f8     eboot.obj
 0001:00000448       ??_C@_0EG@GKGGEOCH@ERROR?3?5ResetDefaultBootCFG?3?5fail@ 00011448     eboot.obj
 0001:00000490       ??_C@_0CP@LKBEOLND@?$AN?6Resetting?5factory?5default?5conf@ 00011490     eboot.obj
 0001:000004c0       ??_C@_07OHKHACFK@0?40?40?40?$AA@ 000114c0     eboot.obj
 0001:000004c8       ??_C@_0CM@PEMGPOKC@INFO?3?5OEMEthSendFrame?3?5retrying?5@ 000114c8     eboot.obj
 0001:000004f4       ??_C@_1BM@MOEMNNDE@?$AAS?$AAa?$AAv?$AAe?$AA?5?$AAS?$AAe?$AAt?$AAt?$AAi?$AAn?$AAg?$AAs?$AA?$AA@ 000114f4     menu.obj
 0001:00000510       ??_C@_1M@PNBPANGG@?$AAR?$AAe?$AAs?$AAe?$AAt?$AA?$AA@ 00011510     menu.obj
 0001:0000051c       ??_C@_1CK@DKDIBGID@?$AAM?$AAM?$AAC?$AA?5?$AAa?$AAn?$AAd?$AA?5?$AAS?$AAD?$AA?5?$AAU?$AAt?$AAi?$AAl?$AAi?$AAt?$AAi?$AAe?$AAs?$AA?$AA@ 0001151c     menu.obj
 0001:00000548       ??_C@_1FC@NIGCHAIH@?$AAL?$AAa?$AAu?$AAn?$AAc?$AAh?$AA?5?$AAE?$AAx?$AAi?$AAs?$AAt?$AAi?$AAn?$AAg?$AA?5?$AAF?$AAl?$AAa?$AAs?$AAh?$AA?5?$AAR?$AAe?$AAs?$AAi?$AAd?$AAe?$AAn?$AAt?$AA?5?$AAI@ 00011548     menu.obj
 0001:0000059c       ??_C@_1CG@PPAMDBLA@?$AAD?$AAo?$AAw?$AAn?$AAl?$AAo?$AAa?$AAd?$AA?5?$AAI?$AAm?$AAa?$AAg?$AAe?$AA?5?$AAN?$AAo?$AAw?$AA?$AA@ 0001159c     menu.obj
 0001:000005c4       ??_C@_1DK@CJENBLML@?$AAS?$AAe?$AAl?$AAe?$AAc?$AAt?$AA?5?$AAW?$AAi?$AAn?$AAd?$AAo?$AAw?$AAs?$AA?5?$AAC?$AAE?$AA?5?$AAD?$AAe?$AAb?$AAu?$AAg?$AA?5?$AAU?$AAA?$AAR?$AAT?$AA?$AA@ 000115c4     menu.obj
 0001:00000600       ??_C@_1CI@MLMJOJI@?$AAS?$AAe?$AAl?$AAe?$AAc?$AAt?$AA?5?$AAE?$AAt?$AAh?$AAe?$AAr?$AA?5?$AAD?$AAe?$AAv?$AAi?$AAc?$AAe?$AA?$AA@ 00011600     menu.obj
 0001:00000628       ??_C@_1CE@PKBKOLCO@?$AAK?$AAI?$AAT?$AAL?$AA?5?$AAP?$AAa?$AAs?$AAs?$AAi?$AAv?$AAe?$AA?5?$AAM?$AAo?$AAd?$AAe?$AA?$AA@ 00011628     menu.obj
 0001:0000064c       ??_C@_1CC@DBLKBKOG@?$AAK?$AAI?$AAT?$AAL?$AA?5?$AAE?$AAn?$AAa?$AAb?$AAl?$AAe?$AA?5?$AAM?$AAo?$AAd?$AAe?$AA?$AA@ 0001164c     menu.obj
 0001:00000670       ??_C@_1BO@PABCHCBJ@?$AAK?$AAI?$AAT?$AAL?$AA?5?$AAW?$AAo?$AAr?$AAk?$AA?5?$AAM?$AAo?$AAd?$AAe?$AA?$AA@ 00011670     menu.obj
 0001:00000690       ??_C@_1CC@PFDHOAOM@?$AAB?$AAo?$AAo?$AAt?$AAl?$AAo?$AAa?$AAd?$AAe?$AAr?$AA?5?$AAS?$AAh?$AAe?$AAl?$AAl?$AA?$AA@ 00011690     menu.obj
 0001:000006b4       ??_C@_1DG@JKEDBFOF@?$AAC?$AAl?$AAe?$AAa?$AAn?$AA?5?$AAr?$AAe?$AAg?$AAi?$AAs?$AAt?$AAr?$AAy?$AA?5?$AA?$CG?$AA?5?$AAd?$AAa?$AAt?$AAa?$AAb?$AAa?$AAs?$AAe?$AAs?$AA?$AA@ 000116b4     menu.obj
 0001:000006ec       ??_C@_1DA@JJAMJFOD@?$AAF?$AAo?$AAr?$AAm?$AAa?$AAt?$AA?5?$AAA?$AAl?$AAl?$AA?5?$AAN?$AAA?$AAN?$AAD?$AA?5?$AAR?$AAe?$AAg?$AAi?$AAo?$AAn?$AAs?$AA?$AA@ 000116ec     menu.obj
 0001:0000071c       ??_C@_1CM@MOIDFHOM@?$AAF?$AAo?$AAr?$AAm?$AAa?$AAt?$AA?5?$AAO?$AAS?$AA?5?$AAN?$AAA?$AAN?$AAD?$AA?5?$AAR?$AAe?$AAg?$AAi?$AAo?$AAn?$AA?$AA@ 0001171c     menu.obj
 0001:00000748       ??_C@_1EO@JEPFIEIH@?$AAR?$AAe?$AAs?$AAe?$AAt?$AA?5?$AAt?$AAo?$AA?5?$AAF?$AAa?$AAc?$AAt?$AAo?$AAr?$AAy?$AA?5?$AAD?$AAe?$AAf?$AAa?$AAu?$AAl?$AAt?$AA?5?$AAC?$AAo?$AAn?$AAf?$AAi?$AAg?$AAu@ 00011748     menu.obj
 0001:00000798       ??_C@_1CG@BBALNGAE@?$AAS?$AAe?$AAl?$AAe?$AAc?$AAt?$AA?5?$AAB?$AAo?$AAo?$AAt?$AA?5?$AAD?$AAe?$AAv?$AAi?$AAc?$AAe?$AA?$AA@ 00011798     menu.obj
 0001:000007c0       ??_C@_1BG@GBKEAKLM@?$AAB?$AAo?$AAo?$AAt?$AA?5?$AAD?$AAe?$AAl?$AAa?$AAy?$AA?$AA@ 000117c0     menu.obj
 0001:000007d8       ??_C@_19DDJNJOGL@?$AAD?$AAH?$AAC?$AAP?$AA?$AA@ 000117d8     menu.obj
 0001:000007e4       ??_C@_1BI@PKAFKBAO@?$AAM?$AAA?$AAC?$AA?5?$AAA?$AAd?$AAd?$AAr?$AAe?$AAs?$AAs?$AA?$AA@ 000117e4     menu.obj
 0001:000007fc       ??_C@_1CA@BMIKHDOB@?$AAS?$AAe?$AAt?$AA?5?$AAM?$AAA?$AAC?$AA?5?$AAA?$AAd?$AAd?$AAr?$AAe?$AAs?$AAs?$AA?$AA@ 000117fc     menu.obj
 0001:0000081c       ??_C@_1BA@LCJJAKKF@?$AAG?$AAa?$AAt?$AAe?$AAw?$AAa?$AAy?$AA?$AA@ 0001181c     menu.obj
 0001:0000082c       ??_C@_1BI@CJHLOJOF@?$AAS?$AAe?$AAt?$AA?5?$AAG?$AAa?$AAt?$AAe?$AAw?$AAa?$AAy?$AA?$AA@ 0001182c     menu.obj
 0001:00000844       ??_C@_1BA@MJOPHPLD@?$AAI?$AAP?$AA?5?$AAM?$AAa?$AAs?$AAk?$AA?$AA@ 00011844     menu.obj
 0001:00000854       ??_C@_1BI@FCANJMPD@?$AAS?$AAe?$AAt?$AA?5?$AAI?$AAP?$AA?5?$AAM?$AAa?$AAs?$AAk?$AA?$AA@ 00011854     menu.obj
 0001:0000086c       ??_C@_1BG@BLDDCHFC@?$AAI?$AAP?$AA?5?$AAA?$AAd?$AAd?$AAr?$AAe?$AAs?$AAs?$AA?$AA@ 0001186c     menu.obj
 0001:00000884       ??_C@_0BC@IHBBJPDE@?5?3?5NK?5from?5NAND?$AN?6?$AA@ 00011884     menu.obj
 0001:00000898       ??_C@_0BE@IIODHDMP@?5?3?5NK?5from?5SD?1MMC?$AN?6?$AA@ 00011898     menu.obj
 0001:000008ac       ??_C@_08HCDDKNJJ@?5?3?5FEC?$AN?6?$AA@ 000118ac     menu.obj
 0001:000008b8       ??_C@_0P@NONOIHBD@?5?3?5USB?5RNDIS?$AN?6?$AA@ 000118b8     menu.obj
 0001:000008c8       ??_C@_0BA@FMMDOFML@?5?3?5USB?5Serial?$AN?6?$AA@ 000118c8     menu.obj
 0001:000008d8       ??_C@_0BE@PKINMFFD@?5?3?5Invalid?5Device?$AN?6?$AA@ 000118d8     menu.obj
 0001:000008ec       ??_C@_0L@CGALPGBD@?5?3?5UART1?$AN?6?$AA@ 000118ec     menu.obj
 0001:000008f8       ??_C@_0L@DELOFJPN@?5?3?5UART2?$AN?6?$AA@ 000118f8     menu.obj
 0001:00000904       ??_C@_0L@IMACDOJI@?5?3?5UART3?$AN?6?$AA@ 00011904     menu.obj
 0001:00000910       ??_C@_0O@CMIFMFKO@?5?3?5Disabled?$AN?6?$AA@ 00011910     menu.obj
 0001:00000920       ??_C@_02PCIJFNDE@?$AN?6?$AA@ 00011920     menu.obj
 0001:00000924       ??_C@_0CH@HJFHFGIJ@INFO?3?5MAC?5address?3?5?$CFx?9?$CFx?9?$CFx?9?$CFx?9?$CF@ 00011924     menu.obj
 0001:00000950       ??_C@_0EA@OMKEPEHK@ERROR?3?5Invalid?5Ethernet?5address?5@ 00011950     menu.obj
 0001:00000990       ??_C@_0CA@OPBDBDDP@?$AN?6Starting?5auto?5download?5?4?4?4?5?$AN?6?$AA@ 00011990     menu.obj
 0001:000009b0       ??_C@_0CA@CLDGGJMD@?$AN?6Launching?5flash?5image?5?5?4?4?4?5?$AN?6?$AA@ 000119b0     menu.obj
 0001:000009d0       ??_C@_0N@FLJDAHIC@?$CFd?5seconds?4?5?$AA@ 000119d0     menu.obj
 0001:000009e0       ??_C@_0EN@KBHLEBPN@?$AN?6Press?5?$FLENTER?$FN?5to?5launch?5image?5@ 000119e0     menu.obj
 0001:00000a30       ??_C@_0EJ@LBCIGPCN@?$AN?6Press?5?$FLENTER?$FN?5to?5launch?5image?5@ 00011a30     menu.obj
 0001:00000a7c       ??_C@_0CK@PCOCDPAP@?$AN?6Initiating?5image?5launch?5in?5?$CFd?5@ 00011a7c     menu.obj
 0001:00000aa8       ??_C@_0DI@JNGDCJGH@?$AN?6Press?5?$FLENTER?$FN?5to?5download?5now?5@ 00011aa8     menu.obj
 0001:00000ae0       ??_C@_0CM@MPOIFBJA@?$AN?6Initiating?5image?5download?5in?5?$CF@ 00011ae0     menu.obj
 0001:00000b10       ??_C@_0EJ@NPNOADG@WARNING?3?5?5Uninitialized?5MAC?5addr@ 00011b10     menu.obj
 0001:00000b5c       ??_C@_0M@CDHNGIPM@?$CFu?4?$CFu?4?$CFu?4?$CFu?$AA@ 00011b5c     oal_blnk:ipformata.obj
 0001:00000b68       ??_C@_1O@INIEDEDF@?$AA?$CI?$AAN?$AAU?$AAL?$AAL?$AA?$CJ?$AA?$AA@ 00011b68     oal_blnk:formata.obj
 0001:00000b78       ??_C@_06LHGEHABH@?$CINULL?$CJ?$AA@ 00011b78     oal_blnk:formata.obj
 0001:00000b80       ??_C@_0CM@HCKAPHGI@ERROR?3?5Failed?5to?5load?5OS?5image?5f@ 00011b80     bootcmn:main.obj
 0001:00000bac       ??_C@_0CN@MKBLLODK@ERROR?3?5Failed?5to?5load?5IPL?5image?5@ 00011bac     bootcmn:main.obj
 0001:00000bdc       ??_C@_0CO@CLCHIGDN@ERROR?3?5Failed?5to?5load?5OS?5image?5f@ 00011bdc     bootcmn:main.obj
 0001:00000c0c       ??_C@_0DB@OPLKFPCH@Received?5boot?5request?5ack?4?4?4?5sta@ 00011c0c     bootcmn:main.obj
 0001:00000c40       ??_C@_0DA@MDAAKDGO@Received?5boot?5request?5ack?4?4?4?5jum@ 00011c40     bootcmn:main.obj
 0001:00000c70       ??_C@_0BO@GOCJJNNJ@Failed?5to?5send?5boot?5request?$AN?6?$AA@ 00011c70     bootcmn:main.obj
 0001:00000c90       ??_C@_0BK@KJKLPNKO@Sending?5boot?5request?4?4?4?$AN?6?$AA@ 00011c90     bootcmn:main.obj
 0001:00000cac       ??_C@_05ENGOENAF@IMX25?$AA@ 00011cac     bootcmn:main.obj
 0001:00000cb4       ??_C@_0BP@KFHIKLKI@INFO?3?5Using?5device?5name?3?5?8?$CFs?8?6?$AA@ 00011cb4     bootcmn:main.obj
 0001:00000cd4       ??_C@_06MHMFDNCL@?$AN?6?$AN?6?$AN?6?$AA@ 00011cd4     bootcmn:main.obj
 0001:00000ce0       ??_C@_0EE@NJJIECID@Download?5successful?$CB?5?5Jumping?5to@ 00011ce0     bootcmn:main.obj
 0001:00000d24       ??_C@_0DA@NOPADPHG@?$AN?6INFO?3?5DIO?5image?5with?5starting?5@ 00011d24     bootcmn:main.obj
 0001:00000d54       ??_C@_0CM@PFPHHIOP@?$AN?6INFO?3?5EBOOT?1SBOOT?5NB0?5remapped@ 00011d54     bootcmn:main.obj
 0001:00000d80       ??_C@_0EK@NNMIMOMC@Specify?5destination?5for?5EBOOT?1SB@ 00011d80     bootcmn:main.obj
 0001:00000dcc       ??_C@_0DN@EFKGNOEL@?$AN?6WARNING?3?5Unsupported?5binary?5fo@ 00011dcc     bootcmn:main.obj
 0001:00000e0c       ??_C@_0CD@BDBOCALK@?$AN?6INFO?3?5NK?5NB0?5remapped?5to?50x?$CFx?4@ 00011e0c     bootcmn:main.obj
 0001:00000e30       ??_C@_0EB@DDOPHGII@Specify?5destination?5for?5NK?5NB0?5?$FL@ 00011e30     bootcmn:main.obj
 0001:00000e74       ??_C@_04IMADAAK@?4nb0?$AA@ 00011e74     bootcmn:main.obj
 0001:00000e7c       ??_C@_09KGAFPJBE@sboot?4nb0?$AA@ 00011e7c     bootcmn:main.obj
 0001:00000e88       ??_C@_09IMLFAILL@eboot?4nb0?$AA@ 00011e88     bootcmn:main.obj
 0001:00000e94       ??_C@_0CD@IJDCBNHD@INFO?3?5XLDR?5NB0?5remapped?5to?50x?$CFx?4@ 00011e94     bootcmn:main.obj
 0001:00000eb8       ??_C@_0EK@CJLNKEGP@Specify?5destination?5for?5XLDR?5NB0@ 00011eb8     bootcmn:main.obj
 0001:00000f04       ??_C@_08NNMHMDLM@xldr?4nb0?$AA@ 00011f04     bootcmn:main.obj
 0001:00000f10       ??_C@_0EF@MBMCDLHM@INFO?3?5OEMMultiBINNotify?5?$CIdwNumRe@ 00011f10     bootcmn:main.obj
 0001:00000f58       ??_C@_0CD@ELMGDNGD@INFO?3?5OEMReportError?5Reason?50x?$CFx@ 00011f58     bootcmn:main.obj
 0001:00000f7c       ??_C@_0CA@OFFHNLCK@ERROR?3?5Invalid?5address?5range?4?$AN?6?$AA@ 00011f7c     bootcmn:main.obj
 0001:00000f9c       ??_C@_0CP@JDGPIHPA@INFO?3?5Downloading?5EBOOT?1SBOOT?5fo@ 00011f9c     bootcmn:main.obj
 0001:00000fcc       ??_C@_0CE@HMABAKKF@INFO?3?5Downloading?5XLDR?5SPI?5image@ 00011fcc     bootcmn:main.obj
 0001:00000ff0       ??_C@_0CL@LNJKHKKB@INFO?3?5Downloading?5XLDR?5I2C?5EEPRO@ 00011ff0     bootcmn:main.obj
 0001:0000101c       ??_C@_0CF@HCMGOJNF@INFO?3?5Downloading?5NK?5SD?1MMC?5imag@ 0001201c     bootcmn:main.obj
 0001:00001044       ??_C@_0DC@PIMDAHJO@INFO?3?5Downloading?5EBOOT?1SBOOT?5fo@ 00012044     bootcmn:main.obj
 0001:00001078       ??_C@_0CH@LGJDEBHD@INFO?3?5Downloading?5XLDR?5SD?1MMC?5im@ 00012078     bootcmn:main.obj
 0001:000010a0       ??_C@_0CC@JCIKJLGP@INFO?3?5Downloading?5NK?5RAM?5image?4?$AN@ 000120a0     bootcmn:main.obj
 0001:000010c4       ??_C@_0CD@CCLLAHMG@INFO?3?5Downloading?5NK?5NAND?5image?4@ 000120c4     bootcmn:main.obj
 0001:000010e8       ??_C@_0CM@BDOCNOGM@INFO?3?5Downloading?5EBOOT?1SBOOT?5NA@ 000120e8     bootcmn:main.obj
 0001:00001114       ??_C@_0CF@KOHMACKP@INFO?3?5Downloading?5XLDR?5NAND?5imag@ 00012114     bootcmn:main.obj
 0001:0000113c       ??_C@_0DO@IAHEPFAH@INFO?3?5OEMVerifyMemory?5?$CICA?5?$DN?50x?$CFx@ 0001213c     bootcmn:main.obj
 0001:0000117c       ??_C@_0CE@PDFEDJGG@INFO?3?5Downloading?5DIO?5NAND?5image@ 0001217c     bootcmn:main.obj
 0001:000011a0       ??_C@_0DG@PBAIANGJ@ERROR?3?5StoreBootCFG?3?5failed?5to?5w@ 000121a0     bootcmn:main.obj
 0001:000011d8       ??_C@_0FG@GFJDGOLO@ERROR?3?5LoadBootCFG?3?5ConfigMagicN@ 000121d8     bootcmn:main.obj
 0001:00001230       ??_C@_0DE@GGGDJLON@ERROR?3?5LoadBootCFG?3?5failed?5to?5lo@ 00012230     bootcmn:main.obj
 0001:00001268       ??_C@_0EL@BJCJJOHF@WARNING?3?5Could?5not?5find?5the?5boot@ 00012268     bootcmn:main.obj
 0001:000012b4       ??_C@_0DI@FJCDBJCA@INFO?3?5OEMPlatformInit?3?5Initializ@ 000122b4     bootcmn:main.obj
 0001:000012f0       ??_C@_0EE@KIMOANOM@WARNING?3?5OEMPlatformInit?3?5Failed@ 000122f0     bootcmn:main.obj
 0001:00001334       ??_C@_0CH@OFHLFLCP@INFO?3?5?5Bootloader?5launched?5from?5@ 00012334     bootcmn:main.obj
 0001:0000135c       ??_C@_0CI@BBFNIMIB@INFO?3?5?5Bootloader?5launched?5from?5@ 0001235c     bootcmn:main.obj
 0001:00001388       ??_C@_0EI@DPIDEJBF@INFO?3?5?5XLDR?5launched?5from?5I2C?5EE@ 00012388     bootcmn:main.obj
 0001:000013d0       ??_C@_0CM@NHECMJBH@INFO?3?5?5Bootloader?5launched?5from?5@ 000123d0     bootcmn:main.obj
 0001:000013fc       ??_C@_0CO@DOGAJLCC@INFO?3?5FAKING?5?5Bootloader?5launche@ 000123fc     bootcmn:main.obj
 0001:00001430       ??_C@_0EA@JPDHBOGB@ERROR?3?5Failed?5to?5initialize?5ARC?5@ 00012430     bootcmn:ether.obj
 0001:00001470       ??_C@_0CK@CODIHID@INFO?3?5Trying?5to?5initialize?5USB?5R@ 00012470     bootcmn:ether.obj
 0001:0000149c       ??_C@_0DH@NMDABBIN@ERROR?3?5Failed?5to?5initialize?5Fast@ 0001249c     bootcmn:ether.obj
 0001:000014d4       ??_C@_0CO@JBGBMPAB@INFO?3?5Fast?5Ethernet?5controller?5i@ 000124d4     bootcmn:ether.obj
 0001:00001504       ??_C@_0DH@HPMFHNO@ERROR?3?5Failed?5to?5initialize?5Fast@ 00012504     bootcmn:ether.obj
 0001:0000153c       ??_C@_0DM@EJPJMAEJ@ERROR?3?5Failed?5to?5initialize?5USB?5@ 0001253c     bootcmn:ether.obj
 0001:00001578       ??_C@_0EC@PJLCGLI@ERROR?3?5Failed?5to?5detect?5and?5init@ 00012578     bootcmn:ether.obj
 0001:000015c0       ??_C@_0EJ@OHBNOOGC@ERROR?3?5Failed?5to?5initialize?5unkn@ 000125c0     bootcmn:ether.obj
 0001:0000160c       ??_C@_0BB@MEBHIIAP@SpinForever?4?4?4?$AN?6?$AA@ 0001260c     bootcmn:utils.obj
 0001:00001620       ??_C@_0BO@LOAGLJOJ@Do?5you?5want?5to?5reset?5?$FLY?2N?$FN?5?$AN?6?$AA@ 00012620     bootcmn:utils.obj
 0001:00001640       ??_C@_0CG@DBIMOJLH@BootTimerInit?3?5EPIT?5mapping?5fail@ 00012640     bootcmn:utils.obj
 0001:00001668       ??_C@_0DF@JLKFBNBO@?$AN?6Enter?5maximum?5number?5of?5second@ 00012668     bootcmn:utils.obj
 0001:000016a0       ??_C@_0CA@PFBHAHMM@Reboot?5the?5device?5manually?4?4?4?$AN?6?$AA@ 000126a0     bootcmn:flash.obj
 0001:000016c0       ??_C@_0CC@GOAJDIEC@Flash?5update?5has?5been?5canceled?4?$AN@ 000126c0     bootcmn:flash.obj
 0001:000016e4       ??_C@_0CG@MMBMGINJ@?$AN?6WARNING?3?5?5Flash?5update?5request@ 000126e4     bootcmn:flash.obj
 0001:0000170c       ??_C@_0CA@IKNJPMAI@Do?5you?5want?5to?5continue?5?$CIy?1n?$CJ?$DP?5?$AA@ 0001270c     bootcmn:flash.obj
 0001:0000172c       ??_C@_0CP@IFDOEFCL@INFO?3?5Update?5of?5XLDR?5completed?5s@ 0001272c     bootcmn:cspi_flash.obj
 0001:0000175c       ??_C@_0CC@DMLNFECM@WARNING?3?5Failed?5to?5verify?5XLDR?4?$AN@ 0001275c     bootcmn:cspi_flash.obj
 0001:00001780       ??_C@_0DB@BAMNCDJA@WARNING?3?5Failed?5to?5read?5XLDR?5in?5@ 00012780     bootcmn:cspi_flash.obj
 0001:000017b4       ??_C@_0CO@MHLLIGAH@WARNING?3?5Failed?5to?5write?5XLDR?5in@ 000127b4     bootcmn:cspi_flash.obj
 0001:000017e4       ??_C@_0CO@OOFAPEAH@WARNING?3?5Unable?5to?5erase?5SPI?5fla@ 000127e4     bootcmn:cspi_flash.obj
 0001:00001818       ??_C@_0EC@IKNNGHEA@INFO?3?5Using?5XLDR?5image?5from?5flas@ 00012818     bootcmn:cspi_flash.obj
 0001:0000185c       ??_C@_0CF@GABMJBPB@ERROR?3?5XLDR?5exceeds?5allocated?5si@ 0001285c     bootcmn:cspi_flash.obj
 0001:00001884       ??_C@_0CO@DBDCEEDI@ERROR?3?5Unable?5to?5get?5SPI?5flash?5i@ 00012884     bootcmn:cspi_flash.obj
 0001:000018b4       ??_C@_0DJ@LJDMMIHA@INFO?3?5Writing?5XLDR?5image?5to?5SPI?5@ 000128b4     bootcmn:cspi_flash.obj
 0001:000018f0       ??_C@_0ED@HJBHPIPI@WARNING?3?5SPI?5Flash?5device?5doesn?8@ 000128f0     bootcmn:cspi_flash.obj
 0001:00001934       ??_C@_0DG@PNOMNNHB@INFO?3?5Update?5of?5EBOOT?1SBOOT?5comp@ 00012934     bootcmn:cspi_flash.obj
 0001:0000196c       ??_C@_0CH@NDFCJD@ERROR?3?5Failed?5to?5verify?5EBOOT?1SB@ 0001296c     bootcmn:cspi_flash.obj
 0001:00001994       ??_C@_0BJ@DHAKPJOJ@INFO?3?5Verifying?5image?4?$AN?6?$AA@ 00012994     bootcmn:cspi_flash.obj
 0001:000019b0       ??_C@_0CH@DLBGIHNI@ERROR?3?5Failed?5to?5update?5EBOOT?1SB@ 000129b0     bootcmn:cspi_flash.obj
 0001:000019d8       ??_C@_0EP@OHKPPMNH@INFO?3?5Programming?5EBOOT?1SBOOT?5im@ 000129d8     bootcmn:cspi_flash.obj
 0001:00001a28       ??_C@_0DB@OLFBJNHF@ERROR?3?5Unable?5to?5erase?5SPI?5flash@ 00012a28     bootcmn:cspi_flash.obj
 0001:00001a5c       ??_C@_0CK@NHLALAMN@INFO?3?5Found?5bad?5SPI?5flash?5block?5@ 00012a5c     bootcmn:cspi_flash.obj
 0001:00001a88       ??_C@_0DA@NIELMACL@INFO?3?5Erasing?5SPI?5flash?5blocks?5?$FL@ 00012a88     bootcmn:cspi_flash.obj
 0001:00001ab8       ??_C@_0DN@HEEIMBBG@ERROR?3?5Boot?5size?5exceeds?5reserve@ 00012ab8     bootcmn:cspi_flash.obj
 0001:00001af8       ??_C@_0DJ@MKEMIADH@INFO?3?5Writing?5Boot?5image?5to?5SPI?5@ 00012af8     bootcmn:cspi_flash.obj
 0001:00001b34       ??_C@_0DN@OKBNDMKM@WARNING?3?5SPI?5device?5doesn?8t?5exis@ 00012b34     bootcmn:cspi_flash.obj
 0001:00001b74       ??_C@_0DE@MHADHDG@ERROR?3?5Failed?5to?5load?5boot?5confi@ 00012b74     bootcmn:cspi_flash.obj
 0001:00001ba8       ??_C@_0CM@KBCPGLLJ@INFO?3?5Loading?5boot?5configuration@ 00012ba8     bootcmn:cspi_flash.obj
 0001:00001bd4       ??_C@_0DG@PDOHILLO@INFO?3?5Successfully?5stored?5boot?5c@ 00012bd4     bootcmn:cspi_flash.obj
 0001:00001c0c       ??_C@_0CB@FMPGMDDB@ERROR?3?5Failed?5to?5update?5EBOOT?4?$AN?6@ 00012c0c     bootcmn:cspi_flash.obj
 0001:00001c30       ??_C@_0CK@EKCHFDOP@INFO?3?5Storing?5boot?5configuration@ 00012c30     bootcmn:cspi_flash.obj
 0001:00001c5c       ??_C@_0CL@BBJPJLKF@ERROR?3?5PageWrite?3?5Write?5EEPROM?5D@ 00012c5c     bootcmn:i2c_eeprom.obj
 0001:00001c88       ??_C@_0CO@HGEGHFHG@ERROR?3?5PageWrite?3?5Write?5EEPROM?5a@ 00012c88     bootcmn:i2c_eeprom.obj
 0001:00001cb8       ??_C@_0CI@CPBFGIJF@ERROR?3?5PageWrite?3?5Generate?5Start@ 00012cb8     bootcmn:i2c_eeprom.obj
 0001:00001ce0       ??_C@_0CJ@FGNAPIED@ERROR?3?5PageRead?3?5Read?5EEPROM?5dat@ 00012ce0     bootcmn:i2c_eeprom.obj
 0001:00001d0c       ??_C@_0CH@PHKPBEHO@ERROR?3?5PageRead?3?5Repeated?5Start?5@ 00012d0c     bootcmn:i2c_eeprom.obj
 0001:00001d34       ??_C@_0CN@IHAHJMEC@ERROR?3?5PageRead?3?5Write?5EEPROM?5ad@ 00012d34     bootcmn:i2c_eeprom.obj
 0001:00001d64       ??_C@_0CH@DKIBMJNB@ERROR?3?5PageRead?3?5Generate?5Start?5@ 00012d64     bootcmn:i2c_eeprom.obj
 0001:00001d90       ??_C@_0EN@EEDEPJBE@ERROR?3?5I2CEEPROMWriteXldr?3?5Read?5@ 00012d90     bootcmn:i2c_eeprom.obj
 0001:00001de0       ??_C@_0CN@OKPHLHJF@ERROR?3?5I2CEEPROMWriteXldr?3?5PageR@ 00012de0     bootcmn:i2c_eeprom.obj
 0001:00001e10       ??_C@_0CO@FJCGKCNG@ERROR?3?5I2CEEPROMWriteXldr?3?5PageW@ 00012e10     bootcmn:i2c_eeprom.obj
 0001:00001e40       ??_C@_0BO@GCKLILNE@ERROR?3?5XLDR?5exceeds?564KByte?$AN?6?$AA@ 00012e40     bootcmn:i2c_eeprom.obj
 0001:00001e60       ??_C@_0CG@MJIEOAAL@I2CEEPROMWriteXldr?3?5dwLength?5?$DN?50@ 00012e60     bootcmn:i2c_eeprom.obj
 0001:00001e88       ??_C@_0CB@KKLHFGEJ@OALStall?3?5EPIT?5mapping?5failed?$CB?$AN?6@ 00012e88     ethdrv:ethdrv.obj
 0001:00001eac       ??_C@_1CI@KDDHFOOJ@?$AAR?$AAe?$AAt?$AAu?$AAr?$AAn?$AA?5?$AAt?$AAo?$AA?5?$AAM?$AAa?$AAi?$AAn?$AA?5?$AAM?$AAe?$AAn?$AAu?$AA?$AA@ 00012eac     blmenu_common_topaz_v1:menu.obj
 0001:00001ed4       ??_C@_1DE@CJJMFMLM@?$AAF?$AAo?$AAr?$AAm?$AAa?$AAt?$AA?5?$AAA?$AAl?$AAl?$AA?5?$AAS?$AAD?$AA?1?$AAM?$AAM?$AAC?$AA?5?$AAR?$AAe?$AAg?$AAi?$AAo?$AAn?$AAs?$AA?$AA@ 00012ed4     blmenu_common_topaz_v1:menu.obj
 0001:00001f08       ??_C@_1GC@OMHINPHG@?$AAC?$AAr?$AAe?$AAa?$AAt?$AAe?$AA?5?$AAF?$AAi?$AAl?$AAe?$AA?5?$AAS?$AAy?$AAs?$AAt?$AAe?$AAm?$AA?5?$AAP?$AAa?$AAr?$AAt?$AAi?$AAt?$AAi?$AAo?$AAn?$AA?5?$AAo?$AAn?$AA?5@ 00012f08     blmenu_common_topaz_v1:menu.obj
 0001:00001f6c       ??_C@_1DI@CHPLHBGN@?$AAe?$AAS?$AAD?$AA?5?$AA2?$AA?4?$AA1?$AA?5?$AAB?$AAo?$AAo?$AAt?$AA?5?$AAP?$AAa?$AAr?$AAt?$AAi?$AAt?$AAi?$AAo?$AAn?$AA?5?$AAS?$AAi?$AAz?$AAe?$AA?$AA@ 00012f6c     blmenu_common_topaz_v1:menu.obj
 0001:00001fa4       ??_C@_1CO@KMCKFBEK@?$AAe?$AAS?$AAD?$AA?5?$AA2?$AA?4?$AA1?$AA?5?$AAB?$AAo?$AAo?$AAt?$AA?5?$AAP?$AAa?$AAr?$AAt?$AAi?$AAt?$AAi?$AAo?$AAn?$AA?$AA@ 00012fa4     blmenu_common_topaz_v1:menu.obj
 0001:00001fd4       ??_C@_1DK@IFGBMPID@?$AAe?$AAM?$AAM?$AAC?$AA?5?$AA4?$AA?4?$AA3?$AA?5?$AAB?$AAo?$AAo?$AAt?$AA?5?$AAP?$AAa?$AAr?$AAt?$AAi?$AAt?$AAi?$AAo?$AAn?$AA?5?$AAS?$AAi?$AAz?$AAe?$AA?$AA@ 00012fd4     blmenu_common_topaz_v1:menu.obj
 0001:00002010       ??_C@_1DA@CKPOEKDC@?$AAe?$AAM?$AAM?$AAC?$AA?5?$AA4?$AA?4?$AA3?$AA?5?$AAB?$AAo?$AAo?$AAt?$AA?5?$AAP?$AAa?$AAr?$AAt?$AAi?$AAt?$AAi?$AAo?$AAn?$AA?$AA@ 00013010     blmenu_common_topaz_v1:menu.obj
 0001:00002040       ??_C@_15JNBOKNOG@?$AA?$AN?$AA?6?$AA?$AA@ 00013040     blmenu_common_topaz_v1:menu.obj
 0001:00002048       ??_C@_15DAMPJCDE@?$AA?$CF?$AAc?$AA?$AA@ 00013048     blmenu_common_topaz_v1:menu.obj
 0001:00002050       ??_C@_17ILCABGPK@?$AA?$AI?$AA?5?$AA?$AI?$AA?$AA@ 00013050     blmenu_common_topaz_v1:menu.obj
 0001:00002058       ??_C@_0N@LPLKOEJA@?5?3?5Enabled?$AN?6?$AA@ 00013058     blmenu_common_topaz_v1:menu.obj
 0001:00002068       ??_C@_0P@LIJBDBHL@?5?3?5?$CFd?5Kbytes?$AN?6?$AA@ 00013068     blmenu_common_topaz_v1:menu.obj
 0001:00002078       ??_C@_0BJ@MGABALLJ@?5?3?5Boot?5and?5r?1w?5part?51?$AN?6?$AA@ 00013078     blmenu_common_topaz_v1:menu.obj
 0001:00002094       ??_C@_0BP@GBDFDBJI@?5?3?5Boot?5part?52?0?5r?1w?5usr?5part?$AN?6?$AA@ 00013094     blmenu_common_topaz_v1:menu.obj
 0001:000020b4       ??_C@_0BJ@NELEKEFH@?5?3?5Boot?5and?5r?1w?5part?52?$AN?6?$AA@ 000130b4     blmenu_common_topaz_v1:menu.obj
 0001:000020d0       ??_C@_0BO@BCOIFLKC@?5?3?5Disabled?5?1?5Not?5Available?$AN?6?$AA@ 000130d0     blmenu_common_topaz_v1:menu.obj
 0001:000020f0       ??_C@_0BP@ILLDOMPK@?5?3?5Boot?5part?51?0?5r?1w?5usr?5part?$AN?6?$AA@ 000130f0     blmenu_common_topaz_v1:menu.obj
 0001:00002110       ??_C@_07LPCKBJPC@Polling?$AA@ 00013110     blmenu_common_topaz_v1:menu.obj
 0001:00002118       ??_C@_09JNFEIGJE@Interrupt?$AA@ 00013118     blmenu_common_topaz_v1:menu.obj
 0001:00002124       ??_C@_07CHEGAGBD@?5?3?5?$CFd?$AN?6?$AA@ 00013124     blmenu_common_topaz_v1:menu.obj
 0001:0000212c       ??_C@_07DOAOMMKG@Enabled?$AA@ 0001312c     blmenu_common_topaz_v1:menu.obj
 0001:00002134       ??_C@_08JGILNPHN@Disabled?$AA@ 00013134     blmenu_common_topaz_v1:menu.obj
 0001:00002140       ??_C@_0BH@IMLFGHDI@?5?3?5?$CFx?9?$CFx?9?$CFx?9?$CFx?9?$CFx?9?$CFx?$AN?6?$AA@ 00013140     blmenu_common_topaz_v1:menu.obj
 0001:00002158       ??_C@_07OKIIGJDF@?5?3?5?$CFs?$AN?6?$AA@ 00013158     blmenu_common_topaz_v1:menu.obj
 0001:00002160       ??_C@_0DC@JJHEEFDO@?$AN?6WARNING?3?5?5Format?5of?5OS?5NAND?5re@ 00013160     blmenu_common_topaz_v1:menu.obj
 0001:00002194       ??_C@_0DE@FMHJGPFH@?$AN?6WARNING?3?5?5Format?5of?5all?5NAND?5r@ 00013194     blmenu_common_topaz_v1:menu.obj
 0001:000021c8       ??_C@_0DP@POLFEJAN@Boot?5loader?5and?5boot?5configurati@ 000131c8     blmenu_common_topaz_v1:menu.obj
 0001:00002208       ??_C@_0CO@BBPEEJNH@ERROR?3?5Unable?5to?5read?5EXT_CSD?5fr@ 00013208     blmenu_common_topaz_v1:menu.obj
 0001:00002238       ??_C@_0DJ@KCKGNILM@?$AN?6WARNING?3?5?5Change?5in?5boot?5parti@ 00013238     blmenu_common_topaz_v1:menu.obj
 0001:00002274       ??_C@_0DH@CLNMIBLA@Data?5on?5all?5partitions?5on?5the?5ca@ 00013274     blmenu_common_topaz_v1:menu.obj
 0001:000022ac       ??_C@_0CM@EGMJHFG@ERROR?3?5Unable?5to?5set?5partition?5a@ 000132ac     blmenu_common_topaz_v1:menu.obj
 0001:000022d8       ??_C@_0DG@NJPLKEB@?$AN?6WARNING?3?5?5Format?5of?5all?5SD?1MMC@ 000132d8     blmenu_common_topaz_v1:menu.obj
 0001:00002310       ??_C@_0ED@JCEMHIBN@Boot?5loader?0?5OS?5and?5boot?5configu@ 00013310     blmenu_common_topaz_v1:menu.obj
 0001:00002358       ??_C@_0HI@PJONFHDK@?$AN?6If?5partition?5creation?5was?5succ@ 00013358     blmenu_common_topaz_v1:menu.obj
 0001:000023d0       ??_C@_0ED@ENHEEIGF@?$AN?6WARNING?3?5?5SD?1MMC?5File?5System?5p@ 000133d0     blmenu_common_topaz_v1:menu.obj
 0001:00002414       ??_C@_0DL@GLMCHJMJ@All?5previous?5file?5system?5data?5on@ 00013414     blmenu_common_topaz_v1:menu.obj
 0001:00002450       ??_C@_19DIEGALPP@?$AA?$CF?$AAc?$AA?$AN?$AA?6?$AA?$AA@ 00013450     blmenu_common_topaz_v1:menu.obj
 0001:0000245c       ??_C@_1BO@MKGCCJBG@?$AA?$AN?$AA?6?$AA?5?$AAS?$AAe?$AAl?$AAe?$AAc?$AAt?$AAi?$AAo?$AAn?$AA?3?$AA?5?$AA?$AA@ 0001345c     blmenu_common_topaz_v1:menu.obj
 0001:0000247c       ??_C@_1BC@NKFMDHEP@?$AA?5?$AA?$FL?$AA?$CF?$AAc?$AA?$FN?$AA?5?$AA?$CF?$AAs?$AA?$AA@ 0001347c     blmenu_common_topaz_v1:menu.obj
 0001:00002490       ??_C@_1BI@MGJPENDP@?$AA?5?$AA?$FL?$AA?$CF?$AAc?$AA?$FN?$AA?5?$AA?$CF?$AAs?$AA?5?$AA?$AN?$AA?6?$AA?$AA@ 00013490     blmenu_common_topaz_v1:menu.obj
 0001:000024a8       ??_C@_1DE@DMLMOHKE@?$AAT?$AAo?$AAp?$AAa?$AAz?$AA?5?$AAi?$AA?4?$AAM?$AAX?$AA2?$AA5?$AA?5?$AAB?$AAo?$AAo?$AAt?$AA?5?$AAM?$AAe?$AAn?$AAu?$AA?5?$AA?$CF?$AAs?$AA?$AA@ 000134a8     blmenu_common_topaz_v1:menu.obj
 0001:000024dc       ??_C@_11LOCGONAA@?$AA?$AA@ 000134dc     blmenu_common_topaz_v1:menu.obj
 0001:000024e0       ??_C@_1CE@DHIEGFHF@?$AA?$CI?$AAU?$AAN?$AAS?$AAA?$AAV?$AAE?$AAD?$AA?5?$AAC?$AAH?$AAA?$AAN?$AAG?$AAE?$AAS?$AA?$CJ?$AA?$AA@ 000134e0     blmenu_common_topaz_v1:menu.obj
 0001:00002508       ??_C@_1KE@LKPJEGMN@?$AA?$AN?$AA?6?$AA?9?$AA?9?$AA?9?$AA?9?$AA?9?$AA?9?$AA?9?$AA?9?$AA?9?$AA?9?$AA?9?$AA?9?$AA?9?$AA?9?$AA?9?$AA?9?$AA?9?$AA?9?$AA?9?$AA?9?$AA?9?$AA?9?$AA?9?$AA?9?$AA?9?$AA?9?$AA?9?$AA?9?$AA?9?$AA?9@ 00013508     blmenu_common_topaz_v1:menu.obj
 0001:000025ac       ??_C@_1CA@IGABMMKB@?$AA?5?$AA?$CF?$AAs?$AA?5?$AAs?$AAe?$AAt?$AA?5?$AAt?$AAo?$AA?5?$AA?$CF?$AAs?$AA?$AN?$AA?6?$AA?$AA@ 000135ac     blmenu_common_topaz_v1:menu.obj
 0001:000025d0       ??_C@_1EA@HMINENJO@?$AA?5?$AA?8?$AA?$CF?$AAs?$AA?8?$AA?5?$AAi?$AAs?$AAn?$AA?8?$AAt?$AA?5?$AAv?$AAa?$AAl?$AAi?$AAd?$AA?5?$AAM?$AAA?$AAC?$AA?5?$AAa?$AAd?$AAd?$AAr?$AAe?$AAs?$AAs?$AA?$AN?$AA?6?$AA?$AA@ 000135d0     blmenu_common_topaz_v1:menu.obj
 0001:00002610       ??_C@_1DA@CFLFOOLN@?$AA?5?$AAE?$AAn?$AAt?$AAe?$AAr?$AA?5?$AA?$CF?$AAs?$AA?5?$AA?$CI?$AAa?$AAc?$AAt?$AAu?$AAa?$AAl?$AA?5?$AA?$CF?$AAs?$AA?$CJ?$AA?3?$AA?5?$AA?$AA@ 00013610     blmenu_common_topaz_v1:menu.obj
 0001:00002640       ??_C@_1DO@PNGPKAIC@?$AA?5?$AA?8?$AA?$CF?$AAs?$AA?8?$AA?5?$AAi?$AAs?$AAn?$AA?8?$AAt?$AA?5?$AAv?$AAa?$AAl?$AAi?$AAd?$AA?5?$AAI?$AAP?$AA?5?$AAa?$AAd?$AAd?$AAr?$AAe?$AAs?$AAs?$AA?$AN?$AA?6?$AA?$AA@ 00013640     blmenu_common_topaz_v1:menu.obj
 0001:00002680       ??_C@_1DI@NFENBBKL@?$AA?5?$AA?8?$AA?$CF?$AAs?$AA?8?$AA?5?$AAi?$AAs?$AAn?$AA?8?$AAt?$AA?5?$AAv?$AAa?$AAl?$AAi?$AAd?$AA?5?$AAI?$AAP?$AA?5?$AAm?$AAa?$AAs?$AAk?$AA?$AN?$AA?6?$AA?$AA@ 00013680     blmenu_common_topaz_v1:menu.obj
 0001:000026b8       ??_C@_0BE@OIKALELC@Unknown?5command?$CB?5?$AN?6?$AA@ 000136b8     bsp_bootshell:bspbootshell.obj
 0001:000026cc       ??_C@_0CJ@BKEGJFOI@Invalid?5parameter?0Please?5Input?5A@ 000136cc     bsp_bootshell:bspbootshell.obj
 0001:000026f8       ??_C@_0M@PDNKHPIC@command?5?9?9?5?$AA@ 000136f8     bsp_bootshell:bspbootshell.obj
 0001:00002704       ??_C@_0DD@HEBPMLJO@?9?9?9?9?9?9?9?9?9?9?9?5?5Topaz?5i?4MX25?5Boot?5S@ 00013704     bsp_bootshell:bspbootshell.obj
 0001:00002738       ??_C@_0BC@JOKBLNPI@type?5?$DP?5for?5help?$AN?6?$AA@ 00013738     bsp_bootshell:bspbootshell.obj
 0001:0000274c       ??_C@_0CI@KMIJHHBB@FECInitDMABuffer?5DMA?5Buffer?5too?5@ 0001374c     oal_ethdrv_fec_common_topaz_v1:fec.obj
 0001:00002774       ??_C@_0CB@DFINIDFK@Failed?5to?5get?5the?5external?5PHY?$AN?6@ 00013774     oal_ethdrv_fec_common_topaz_v1:fec.obj
 0001:00002798       ??_C@_0CN@NECAPPEM@FEC?5is?5linked?0?5speed?510?5Mbps?0?5ha@ 00013798     oal_ethdrv_fec_common_topaz_v1:fec.obj
 0001:000027c8       ??_C@_0CN@KMHKLMCP@FEC?5is?5linked?0?5speed?510?5Mbps?0?5fu@ 000137c8     oal_ethdrv_fec_common_topaz_v1:fec.obj
 0001:000027f8       ??_C@_0CO@NCDNBHO@FEC?5is?5linked?0?5speed?5100?5Mbps?0?5h@ 000137f8     oal_ethdrv_fec_common_topaz_v1:fec.obj
 0001:00002828       ??_C@_0CO@HFHJJCBN@FEC?5is?5linked?0?5speed?5100?5Mbps?0?5f@ 00013828     oal_ethdrv_fec_common_topaz_v1:fec.obj
 0001:00002858       ??_C@_0BL@PCLOMCF@Initializing?5Ethernet?4?4?4?$AN?6?$AA@ 00013858     oal_ethdrv_fec_common_topaz_v1:fec.obj
 0001:00002874       ??_C@_0BK@FGOBGFEM@RNDISMINI?5?9?9?9?5RESET?5?9?9?9?$AN?6?$AA@ 00013874     fsl_rne_mdd_common_topaz_v1:rndis.obj
 0001:00002890       ??_C@_0CK@HCFNMAPL@RNdis?3?3?5Too?5much?5outgoing?0?5baili@ 00013890     fsl_rne_mdd_common_topaz_v1:rndis.obj
 0001:000028bc       ??_C@_0DK@LOJODLJL@ASSERT?$CB?5Rndis?3?3MddSendRndisMessa@ 000138bc     fsl_rne_mdd_common_topaz_v1:rndis.obj
 0001:000028f8       ??_C@_0DI@ELIDGGNF@ASSERT?5Fail?5at?5uiMessageSize?$CI?$CFd?$CJ@ 000138f8     fsl_rne_mdd_common_topaz_v1:rndis.obj
 0001:00002930       ??_C@_0CK@BEACHKGH@RNdis?3?3?5No?5mem?5for?5INITIALIZE_CO@ 00013930     fsl_rne_mdd_common_topaz_v1:rndis.obj
 0001:0000295c       ??_C@_0BN@MJFOLLBM@RNdis?3?3?5Should?5not?5happen?$CB?$AN?6?$AA@ 0001395c     fsl_rne_mdd_common_topaz_v1:rndis.obj
 0001:0000297c       ??_C@_0CO@JHJMPDCG@RNDISMINI?5Err?$CB?$CB?5unsupported?5RNDI@ 0001397c     fsl_rne_mdd_common_topaz_v1:rndis.obj
 0001:000029ac       ??_C@_0CP@HEPIJLKK@RndisMdd?3?3?5PDD?8s?5max?5RX?5buffer?5?$DN@ 000139ac     fsl_rne_mdd_common_topaz_v1:rndis.obj
 0001:000029dc       ??_C@_0CK@JCOPOCLM@ERROR?$CB?5RndisInitialize?5msg?5recei@ 000139dc     fsl_rne_mdd_common_topaz_v1:rndis.obj
 0001:00002a08       ??_C@_0DB@NGCDHJGD@RndisMini?5recv?5REMOTE_NDIS_HALT_@ 00013a08     fsl_rne_mdd_common_topaz_v1:rndis.obj
 0001:00002a3c       ??_C@_09JBPNJICM@rndis?4cpp?$AA@ 00013a3c     fsl_rne_mdd_common_topaz_v1:rndis.obj
 0001:00002a48       ??_C@_0BP@HHOMIKAO@ASSERT?5at?5File?$CI?$CFs?$CJ?5line?5?$CI?$CFd?$CJ?$AN?6?$AA@ 00013a48     fsl_rne_mdd_common_topaz_v1:rndis.obj
 0001:00002a68       ??_C@_0DB@PAFHLFPB@RndisMini?5rcv?5REMOTE_NDIS_RESET_@ 00013a68     fsl_rne_mdd_common_topaz_v1:rndis.obj
 0001:00002a9c       ??_C@_0DA@CMCBBBCA@RNdis?3?3?5Unknown?5RNDIS?5msg?0?5buff?$FL@ 00013a9c     fsl_rne_mdd_common_topaz_v1:rndis.obj
 0001:00002acc       ??_C@_0P@BDJJIKDL@Overrun?$DN0x?$CFx?6?$AN?$AA@ 00013acc     fsl_rne_mdd_common_topaz_v1:rndis.obj
 0001:00002adc       ??_C@_0BJ@IJMDONAK@Buffer?5is?5too?5big?50x?$CFx?6?$AN?$AA@ 00013adc     fsl_rne_mdd_common_topaz_v1:rndis.obj
 0001:00002af8       ??_C@_0CK@LKMHPIGI@Wrong?5Data?5DataLength?5Msg?$DN0x?$CFx?0P@ 00013af8     fsl_rne_mdd_common_topaz_v1:rndis.obj
 0001:00002b24       ??_C@_0CN@OHNGADLJ@RNdis?3?3?5Invalid?5RndisPacket?5l?$FL?$CFd@ 00013b24     fsl_rne_mdd_common_topaz_v1:rndis.obj
 0001:00002b54       ??_C@_0BH@HBKBIINO@Wrong?5Data?5Type?50x?$CFx?$AN?6?$AA@ 00013b54     fsl_rne_mdd_common_topaz_v1:rndis.obj
 0001:00002b6c       ??_C@_0CA@IBGOHNCO@Rndis?3?3?5initialization?3?5Fail?$CB?$AN?6?$AA@ 00013b6c     fsl_rne_mdd_common_topaz_v1:rndis.obj
 0001:00002b8c       ??_C@_0CC@EELLDCCI@Rndis?3?3?5initialization?3?5Success?$AN@ 00013b8c     fsl_rne_mdd_common_topaz_v1:rndis.obj
 0001:00002bb0       ??_C@_0CD@EOFHIDOL@Rndis?3?3?5Get?5MAC?5address?5?$CFx?0?$CFx?0?$CFx@ 00013bb0     fsl_rne_mdd_common_topaz_v1:rndis.obj
 0001:00002bd4       ??_C@_0CM@KLOLOCDD@Rndis?3?3?5Err?5no?5MAC?5address?5read?5@ 00013bd4     fsl_rne_mdd_common_topaz_v1:rndis.obj
 0001:00002c00       ??_C@_0BL@EINAHMEI@Rndis?3?3?5PDDInit?5Success?$CB?$AN?6?$AA@ 00013c00     fsl_rne_mdd_common_topaz_v1:rndis.obj
 0001:00002c1c       ??_C@_0BK@BFGGBGMH@Rndis?3?3?5initialization?$CB?$AN?6?$AA@ 00013c1c     fsl_rne_mdd_common_topaz_v1:rndis.obj
 0001:00002c38       ??_C@_0CI@PFDJABBD@Rndis?3?3?5Address?5static?5map?5to?5ad@ 00013c38     fsl_rne_mdd_common_topaz_v1:rndis.obj
 0001:00002c60       ??_C@_0CH@LBCKJEJO@Rndis?3?3?5initialization?3?5with?5add@ 00013c60     fsl_rne_mdd_common_topaz_v1:rndis.obj
 0001:00002c88       ??_C@_0BP@JDIDIKNB@OID?$FL?$CFx?$FN?5not?5yet?5implemented?$CB?$AN?6?$AA@ 00013c88     fsl_rne_mdd_common_topaz_v1:hostmini.obj
 0001:00002ca8       ??_C@_0CP@MKNOHPIM@HostMini?3?3?5New?5filter?5set?3?5?$FL0x?$CFx@ 00013ca8     fsl_rne_mdd_common_topaz_v1:hostmini.obj
 0001:00002cd8       ??_C@_0BE@LPGPNKBH@HostMiniInit?3?3?5?$CB?$CB?$AN?6?$AA@ 00013cd8     fsl_rne_mdd_common_topaz_v1:hostmini.obj
 0001:00002cec       ??_C@_1O@NJEHEHHO@?$AAu?$AAt?$AAi?$AAl?$AA?4?$AAc?$AA?$AA@ 00013cec     fsl_rne_mdd_common_topaz_v1:util.obj
 0001:00002d00       ??_C@_1FA@PHGBNLGM@?$AAM?$AAi?$AAc?$AAr?$AAo?$AAs?$AAo?$AAf?$AAt?$AA?5?$AAR?$AAN?$AAD?$AAI?$AAS?$AA?5?$AAK?$AAI?$AAT?$AAL?$AA?5?$AAf?$AAo?$AAr?$AA?5?$AAF?$AAS?$AAL?$AA?5?$AAH?$AAS?$AA?5@ 00013d00     fsl_rne_pdd_common_topaz_v1:rndis_pdd.obj
 0001:00002d50       ??_C@_1BE@DEAPIJA@?$AAM?$AAi?$AAc?$AAr?$AAo?$AAs?$AAo?$AAf?$AAt?$AA?$AA@ 00013d50     fsl_rne_pdd_common_topaz_v1:rndis_pdd.obj
 0001:00002d78       DigitTable                 00013d78     fsl_rne_pdd_common_topaz_v1:rndis_pdd.obj
 0001:00002d9c       ??_C@_0BO@FJNCJEJP@Discard?5?$CFd?5Pending?5Messages?$AN?6?$AA@ 00013d9c     fsl_rne_pdd_common_topaz_v1:rndis_pdd.obj
 0001:00002dbc       ??_C@_1BC@GDFGLIEL@?$AAO?$AAT?$AAG?$AAG?$AAr?$AAo?$AAu?$AAp?$AA?$AA@ 00013dbc     usb_usbfn_mx25_topaz_v1:i_pdd.obj
 0001:00002dd0       ??_C@_1BG@HHFAGDDC@?$AAO?$AAT?$AAG?$AAS?$AAu?$AAp?$AAp?$AAo?$AAr?$AAt?$AA?$AA@ 00013dd0     usb_usbfn_mx25_topaz_v1:i_pdd.obj
 0001:00002de8       ??_C@_1BI@BHLBGEOK@?$AAP?$AAr?$AAi?$AAo?$AAr?$AAi?$AAt?$AAy?$AA2?$AA5?$AA6?$AA?$AA@ 00013de8     usb_usbfn_mx25_topaz_v1:i_pdd.obj
 0001:00002e00       ??_C@_17DJGGJCGD@?$AAI?$AAr?$AAq?$AA?$AA@ 00013e00     usb_usbfn_mx25_topaz_v1:i_pdd.obj
 0001:00002e08       ??_C@_1O@LBBNFMDB@?$AAM?$AAe?$AAm?$AAL?$AAe?$AAn?$AA?$AA@ 00013e08     usb_usbfn_mx25_topaz_v1:i_pdd.obj
 0001:00002e18       ??_C@_1BA@INLDIDEN@?$AAM?$AAe?$AAm?$AAB?$AAa?$AAs?$AAe?$AA?$AA@ 00013e18     usb_usbfn_mx25_topaz_v1:i_pdd.obj
 0001:00002eb8       ??_C@_1BM@LGGJJGMB@?$AAP?$AAr?$AAi?$AAm?$AAe?$AAF?$AAZ?$AAL?$AAT?$AA?3?$AA?5?$AA?$CF?$AAs?$AA?$AA@ 00013eb8     usb_usbfn_mx25_topaz_v1:i_pdd.obj
 0001:00002ed4       ??_C@_17HCEMPBGG@?$AAO?$AAU?$AAT?$AA?$AA@ 00013ed4     usb_usbfn_mx25_topaz_v1:i_pdd.obj
 0001:00002edc       ??_C@_15BNKBCKPG@?$AAI?$AAN?$AA?$AA@ 00013edc     usb_usbfn_mx25_topaz_v1:i_pdd.obj
 0001:00002ee8       ??_C@_1EA@GOCNCOIC@?$AAI?$AAs?$AAs?$AAu?$AAe?$AAT?$AAr?$AAa?$AAn?$AAs?$AAf?$AAe?$AAr?$AA?3?$AA?5?$AA?$CF?$AAs?$AA?5?$AAw?$AAi?$AAt?$AAh?$AA?5?$AA?$CF?$AAd?$AA?5?$AAb?$AAy?$AAt?$AAe?$AAs?$AA?$AA@ 00013ee8     usb_usbfn_mx25_topaz_v1:i_pdd.obj
 0001:00002f28       ??_C@_1DA@JMEFNML@?$AAA?$AAb?$AAo?$AAr?$AAt?$AAT?$AAr?$AAa?$AAn?$AAs?$AAf?$AAe?$AAr?$AA?5?$AA?$CI?$AA?$CF?$AAs?$AA?5?$AAE?$AAP?$AA?$CF?$AAd?$AA?$CJ?$AA?$AA@ 00013f28     usb_usbfn_mx25_topaz_v1:i_pdd.obj
 0001:00002f58       ??_C@_19CIJIHAKK@?$AAN?$AAU?$AAL?$AAL?$AA?$AA@ 00013f58     usb_usbfn_mx25_topaz_v1:i_pdd.obj
 0001:00002f64       ??_C@_1CA@HMLLGPGC@?$AA?9?$AAS?$AAe?$AAn?$AAd?$AAC?$AAS?$AAH?$AA?5?$AA?$CI?$AAE?$AAP?$AA?$CF?$AAd?$AA?$CJ?$AA?$AA@ 00013f64     usb_usbfn_mx25_topaz_v1:i_pdd.obj
 0001:00002f84       ??_C@_1CA@DFPEHIFN@?$AA?$CL?$AAS?$AAe?$AAn?$AAd?$AAC?$AAS?$AAH?$AA?5?$AA?$CI?$AAE?$AAP?$AA?$CF?$AAd?$AA?$CJ?$AA?$AA@ 00013f84     usb_usbfn_mx25_topaz_v1:i_pdd.obj
 0001:00002fa4       ??_C@_1CI@HKDMKLGF@?$AAD?$AAe?$AAt?$AAa?$AAc?$AAh?$AA?3?$AA?5?$AAP?$AAO?$AAR?$AAT?$AAS?$AAC?$AA?5?$AA0?$AAx?$AA?$CF?$AAx?$AA?$AA@ 00013fa4     usb_usbfn_mx25_topaz_v1:i_pdd.obj
 0001:00002fcc       ??_C@_1O@BJIMCIMK@?$AAR?$AAe?$AAs?$AAu?$AAm?$AAe?$AA?$AA@ 00013fcc     usb_usbfn_mx25_topaz_v1:i_pdd.obj
 0001:00002fdc       ??_C@_1BE@JNFMNJIM@?$AAI?$AAn?$AAt?$AAr?$AA?3?$AAD?$AAo?$AAn?$AAe?$AA?$AA@ 00013fdc     usb_usbfn_mx25_topaz_v1:i_pdd.obj
 0001:00002ff0       ??_C@_1EE@JAFGGGNF@?$AAI?$AAn?$AAt?$AAr?$AA?3?$AAU?$AAI?$AA?5?$AAS?$AAE?$AAT?$AAU?$AAP?$AAS?$AAT?$AAA?$AAT?$AA?5?$AA?$CF?$AAx?$AA?5?$AAE?$AAN?$AAD?$AAP?$AAT?$AAC?$AAO?$AAM?$AAP?$AA?5?$AA?$CF@ 00013ff0     usb_usbfn_mx25_topaz_v1:i_pdd.obj
 0001:00003034       ??_C@_1BC@MCOFDLFC@?$AAI?$AAn?$AAt?$AAr?$AA?3?$AAS?$AAL?$AAI?$AA?$AA@ 00014034     usb_usbfn_mx25_topaz_v1:i_pdd.obj
 0001:00003048       ??_C@_1BO@EGKDOEEI@?$AAI?$AAn?$AAt?$AAr?$AA?3?$AAS?$AAi?$AAg?$AAn?$AAa?$AAl?$AAl?$AAe?$AAd?$AA?$AA@ 00014048     usb_usbfn_mx25_topaz_v1:i_pdd.obj
 0001:0000306c       ??_C@_0CA@LIHOEDHI@failed?5to?5receive?5header?5data?$AN?6?$AA@ 0001406c     oal_blserial:serfuncs.obj
 0001:0000308c       ??_C@_0BH@MJPKDDID@header?5checksum?5fail?$AN?6?$AA@ 0001408c     oal_blserial:serfuncs.obj
 0001:000030a4       ??_C@_0CF@PODCGAIM@failed?5to?5receive?5header?5signatu@ 000140a4     oal_blserial:serfuncs.obj
 0001:000030cc       ??_C@_0CJ@CHGIGMLG@received?5non?9download?5packet?5typ@ 000140cc     oal_blserial:serfuncs.obj
 0001:000030f8       ??_C@_0DG@MLEBFPEB@data?5checksum?5failure?4?5expected?5@ 000140f8     oal_blserial:serfuncs.obj
 0001:00003130       ??_C@_0BN@FEFEJPIP@failed?5to?5read?5packet?5data?$AN?6?$AA@ 00014130     oal_blserial:serfuncs.obj
 0001:00003150       ??_C@_0CM@DECDFMCF@insufficient?5buffer?5size?$DL?5ignori@ 00014150     oal_blserial:serfuncs.obj
 0001:0000317c       ??_C@_0BL@MMGBDAGN@failed?5to?5receive?5header?$AN?6?$AA@ 0001417c     oal_blserial:serfuncs.obj
 0001:00003198       ??_C@_0CE@HOCBBCP@Received?5out?5of?5sequence?5block?5?$CF@ 00014198     oal_blserial:serfuncs.obj
 0001:000031bc       ??_C@_0BE@KEIPDPMM@Expected?5block?5?$CFu?$AN?6?$AA@ 000141bc     oal_blserial:serfuncs.obj
 0001:000031d0       ??_C@_0BK@IPKIMKPH@Waiting?5for?5boot?5ack?4?4?4?$AN?6?$AA@ 000141d0     oal_blserial:serfuncs.obj
 0001:000031ec       ??_C@_0CK@DMEOPGMB@Got?5jump?5request?0?5KITL?5transport@ 000141ec     oal_blserial:serfuncs.obj
 0001:00003218       ??_C@_0CM@FEMLNPOM@ERROR?3?5Unable?5to?5set?5block?5statu@ 00014218     nand_boot_common_topaz_v1:nandboot.obj
 0001:00003244       ??_C@_0DC@FINGMGAN@ERROR?3?5Unable?5to?5erase?5NAND?5flas@ 00014244     nand_boot_common_topaz_v1:nandboot.obj
 0001:00003278       ??_C@_0CL@JNFABMJO@INFO?3?5Found?5bad?5NAND?5flash?5block@ 00014278     nand_boot_common_topaz_v1:nandboot.obj
 0001:000032a4       ??_C@_0BN@PPPNLHLF@WARNING?3?5NANDBootInit?5fail?$AN?6?$AA@ 000142a4     nand_boot_common_topaz_v1:nandboot.obj
 0001:000032c4       ??_C@_0CP@MEMGALMB@ERROR?3?5Unable?5to?5get?5NAND?5flash?5@ 000142c4     nand_boot_common_topaz_v1:nandboot.obj
 0001:000032f4       ??_C@_0BO@PPFGHOP@ERROR?3?5Failed?5to?5verify?5NK?4?$AN?6?$AA@ 000142f4     nand_boot_common_topaz_v1:nandboot.obj
 0001:00003314       ??_C@_0DC@BCKCJKFP@WARNING?3?5Failed?5to?5write?5XLDR?5in@ 00014314     nand_boot_common_topaz_v1:nandboot.obj
 0001:00003348       ??_C@_0DG@BACIOMAB@Error?3?5No?5good?5block?5found?5?9?5una@ 00014348     nand_boot_common_topaz_v1:nandboot.obj
 0001:00003380       ??_C@_0DO@KAJJOHBJ@ERROR?3?5XLDR?5size?5exceeds?5reserve@ 00014380     nand_boot_common_topaz_v1:nandboot.obj
 0001:000033c0       ??_C@_0DE@DHNKGOFC@INFO?3?5Writing?5XLDR?5image?5to?5NAND@ 000143c0     nand_boot_common_topaz_v1:nandboot.obj
 0001:000033f4       ??_C@_0DO@NAFJLJJO@WARNING?3?5NAND?5device?5doesn?8t?5exi@ 000143f4     nand_boot_common_topaz_v1:nandboot.obj
 0001:00003434       ??_C@_0CB@PJJBOHIF@INFO?3?5Verifying?5image?5succeed?4?$AN?6@ 00014434     nand_boot_common_topaz_v1:nandboot.obj
 0001:00003458       ??_C@_0DO@IACNLFIB@INFO?3?5Updating?5of?5EBOOT?1SBOOT?5im@ 00014458     nand_boot_common_topaz_v1:nandboot.obj
 0001:00003498       ??_C@_0CL@HLKKIBHF@NAND?5flash?5block?5?$FL0x?$CFx?$FN?5isn?8t?5re@ 00014498     nand_boot_common_topaz_v1:nandboot.obj
 0001:000034c4       ??_C@_0CB@COMIICDO@ERROR?3?5Failed?5to?5verify?5image?4?$AN?6@ 000144c4     nand_boot_common_topaz_v1:nandboot.obj
 0001:000034e8       ??_C@_0DF@DMMPELAE@INFO?3?5Programming?5NAND?5flash?5blo@ 000144e8     nand_boot_common_topaz_v1:nandboot.obj
 0001:00003520       ??_C@_0DO@LHIODLEE@ERROR?3?5Boot?5size?5exceeds?5reserve@ 00014520     nand_boot_common_topaz_v1:nandboot.obj
 0001:00003560       ??_C@_0DE@DFOAOGPK@INFO?3?5Writing?5Boot?5image?5to?5NAND@ 00014560     nand_boot_common_topaz_v1:nandboot.obj
 0001:00003594       ??_C@_0CD@LBDDECMN@?$AN?6INFO?3?5Verifying?5image?5succeed?4@ 00014594     nand_boot_common_topaz_v1:nandboot.obj
 0001:000035b8       ??_C@_0DC@BGNPKHBI@INFO?3?5Updating?5of?5image?5complete@ 000145b8     nand_boot_common_topaz_v1:nandboot.obj
 0001:000035ec       ??_C@_0CB@PAFJJGNA@ERROR?3?5Failed?5to?5update?5image?4?$AN?6@ 000145ec     nand_boot_common_topaz_v1:nandboot.obj
 0001:00003610       ??_C@_0DK@BNDNAAAI@INFO?3?5Programming?5and?5Verifying?5@ 00014610     nand_boot_common_topaz_v1:nandboot.obj
 0001:0000364c       ??_C@_0DF@NNJDPACB@INFO?3?5Programming?5NAND?5flash?5blo@ 0001464c     nand_boot_common_topaz_v1:nandboot.obj
 0001:00003684       ??_C@_0DM@FFNMNECJ@ERROR?3?5NK?5size?5exceeds?5reserved?5@ 00014684     nand_boot_common_topaz_v1:nandboot.obj
 0001:000036c0       ??_C@_0DC@IBLKHNEB@INFO?3?5Writing?5NK?5image?5to?5NAND?5?$CI@ 000146c0     nand_boot_common_topaz_v1:nandboot.obj
 0001:000036f4       ??_C@_0DA@CFIHFKOJ@?$AN?6INFO?3?5Loading?5of?5NK?5completed?5@ 000146f4     nand_boot_common_topaz_v1:nandboot.obj
 0001:00003724       ??_C@_0CF@PLBLFIAH@ERROR?3?5Read?5sector?3?5?$FL0x?$CFx?$FN?5faile@ 00014724     nand_boot_common_topaz_v1:nandboot.obj
 0001:0000374c       ??_C@_02GPIOPFAK@?$DO?$DO?$AA@ 0001474c     nand_boot_common_topaz_v1:nandboot.obj
 0001:00003750       ??_C@_0DC@PEELBEJC@INFO?3?5Reading?5NK?5image?5to?5NAND?5?$CI@ 00014750     nand_boot_common_topaz_v1:nandboot.obj
 0001:00003784       ??_C@_0DN@FOBINPEN@WARNING?3?5NAND?5device?5doesn?8t?5exi@ 00014784     nand_boot_common_topaz_v1:nandboot.obj
 0001:000037c4       ??_C@_0CO@BJGFJAIH@WARNING?3?5Failed?5to?5Load?5configur@ 000147c4     nand_boot_common_topaz_v1:nandboot.obj
 0001:000037f4       ??_C@_0BO@PCFMGLDF@Error?3?5No?5good?5block?5found?$CB?$AN?6?$AA@ 000147f4     nand_boot_common_topaz_v1:nandboot.obj
 0001:00003814       ??_C@_0CN@NHADDNNL@INFO?3?5Loading?5boot?5configuration@ 00014814     nand_boot_common_topaz_v1:nandboot.obj
 0001:00003844       ??_C@_0DI@OLNJMAJP@INFO?3?5Successfully?5stored?5boot?5c@ 00014844     nand_boot_common_topaz_v1:nandboot.obj
 0001:0000387c       ??_C@_0DE@LLENDJKK@WARNING?3?5Failed?5to?5write?5boot?5co@ 0001487c     nand_boot_common_topaz_v1:nandboot.obj
 0001:000038b0       ??_C@_0DJ@HCHCAAAK@INFO?3?5Storing?5boot?5configuration@ 000148b0     nand_boot_common_topaz_v1:nandboot.obj
 0001:000038f0       ??_C@_0ED@HDAKJGJP@Error?3?5No?5good?5block?5found?5?9?5una@ 000148f0     nand_boot_common_topaz_v1:nandboot.obj
 0001:00003934       ??_C@_0DL@JLHJEAKF@?$AN?6INFO?3?5Format?5of?5NAND?5NK?5region@ 00014934     nand_boot_common_topaz_v1:nandboot.obj
 0001:00003970       ??_C@_0CL@OKPLEKII@INFO?3?5Starting?5format?5of?5NAND?5NK@ 00014970     nand_boot_common_topaz_v1:nandboot.obj
 0001:0000399c       ??_C@_0CO@FFMLABON@INFO?3?5Update?5of?5IPL?5completed?5su@ 0001499c     nand_boot_common_topaz_v1:nandboot.obj
 0001:000039cc       ??_C@_0BP@DCNJBMKK@ERROR?3?5Failed?5to?5verify?5IPL?4?$AN?6?$AA@ 000149cc     nand_boot_common_topaz_v1:nandboot.obj
 0001:000039f0       ??_C@_0EH@DDGBHFHG@INFO?3?5Programming?5IPL?5image?5from@ 000149f0     nand_boot_common_topaz_v1:nandboot.obj
 0001:00003a38       ??_C@_0DN@MHDNDODE@ERROR?3?5IPL?5size?5exceeds?5reserved@ 00014a38     nand_boot_common_topaz_v1:nandboot.obj
 0001:00003a78       ??_C@_0DD@FBNOANAB@INFO?3?5Writing?5IPL?5image?5to?5NAND?5@ 00014a78     nand_boot_common_topaz_v1:nandboot.obj
 0001:00003aac       ??_C@_0CI@KOKADIKC@?$AN?6INFO?3?5Ready?5to?5write?5DIO?5image@ 00014aac     nand_boot_common_topaz_v1:nandboot.obj
 0001:00003ad4       ??_C@_0BO@IMFCJLLN@INFO?3?5Erase?5is?5?$CFd?$CF?$CF?5complete?4?$AA@ 00014ad4     nand_boot_common_topaz_v1:nandboot.obj
 0001:00003af4       ??_C@_0DB@NKJDIEPK@INFO?3?5Erasing?5NAND?5flash?5blocks?5@ 00014af4     nand_boot_common_topaz_v1:nandboot.obj
 0001:00003b28       ??_C@_0ED@JNNBGIKF@ERROR?3?5DIO?5image?5size?5exceeds?5re@ 00014b28     nand_boot_common_topaz_v1:nandboot.obj
 0001:00003b70       ??_C@_0ED@MCLEPO@ERROR?3?5Incorrect?5or?5corrupted?5DI@ 00014b70     nand_boot_common_topaz_v1:nandboot.obj
 0001:00003bb8       ??_C@_0EG@LILMDEGK@WARN?3?5Block?5?$FL0x?$CFx?$FN?5?1?5sector?5?$FL0x?$CF@ 00014bb8     nand_boot_common_topaz_v1:nandboot.obj
 0001:00003c00       ??_C@_0CH@DAJMGFOB@ERROR?3?5Writing?5sector?5?$FL0x?$CFx?$FN?5fai@ 00014c00     nand_boot_common_topaz_v1:nandboot.obj
 0001:00003c28       ??_C@_0DG@POHOAOBL@?$AN?6INFO?3?5Update?5of?5DIO?5image?5comp@ 00014c28     nand_boot_common_topaz_v1:nandboot.obj
 0001:00003c60       ??_C@_0BL@KGENHFNE@?$AN?6INFO?3?5No?5NAND?5present?$CB?$AN?6?$AA@ 00014c60     nand_boot_common_topaz_v1:nandboot.obj
 0001:00003c7c       ??_C@_0CM@MAKCJGJN@INFO?3?5Copy?5of?5IPL?5completed?5succ@ 00014c7c     nand_boot_common_topaz_v1:nandboot.obj
 0001:00003ca8       ??_C@_0CO@DIGEHKBF@INFO?3?5Copying?5IPL?5image?5to?5RAM?5a@ 00014ca8     nand_boot_common_topaz_v1:nandboot.obj
 0001:00003cd8       ??_C@_0DF@OLHDGLNN@INFO?3?5Reading?5IPL?5image?5from?5NAN@ 00014cd8     nand_boot_common_topaz_v1:nandboot.obj
 0001:00003d10       ??_C@_0DN@CCBKKGDF@?$AN?6INFO?3?5Format?5of?5all?5NAND?5regio@ 00014d10     nand_boot_common_topaz_v1:nandboot.obj
 0001:00003d50       ??_C@_0BP@HLOCHMLD@INFO?3?5Format?5is?5?$CFd?$CF?$CF?5complete?4?$AA@ 00014d50     nand_boot_common_topaz_v1:nandboot.obj
 0001:00003d70       ??_C@_0DA@GHJFJAN@ERROR?3?5Unable?5to?5erase?5NAND?5flas@ 00014d70     nand_boot_common_topaz_v1:nandboot.obj
 0001:00003da0       ??_C@_0CN@CCDNFIGE@INFO?3?5Starting?5format?5of?5all?5NAN@ 00014da0     nand_boot_common_topaz_v1:nandboot.obj
 0001:00003e50       ??_C@_0BK@BFELHAIB@EthDown?3?3TFTPD_OPEN?3?3?$CFs?$AN?6?$AA@ 00014e50     eboot:ebsimp.obj
 0001:00003e6c       ??_C@_0CF@NJGKJDPK@EthDown?3?3Illegal?5Operation?5Code?5@ 00014e6c     eboot:ebsimp.obj
 0001:00003e94       ??_C@_0BN@HCIGGCJK@Server?5Registration?5Failed?$AN?6?$AA@ 00014e94     eboot:ebsimp.obj
 0001:00003eb4       ??_C@_0CC@OIEKENJI@EbootSimpleTFTP?5not?5initialized?$AN@ 00014eb4     eboot:ebsimp.obj
 0001:00003ed8       ??_C@_0BM@GELEBJHM@EbootGratuitousARP?5failed?$AN?6?$AA@ 00014ed8     eboot:ebsimp.obj
 0001:00003ef4       ??_C@_0DG@LCJHGIIG@Some?5other?5station?5has?5IP?5Addres@ 00014ef4     eboot:ebsimp.obj
 0001:00003f2c       ??_C@_0DK@ECECEHHP@No?5ARP?5response?5in?5?$CFd?5seconds?0?5a@ 00014f2c     eboot:ebsimp.obj
 0001:00003f68       ??_C@_0CO@EJPPGFNA@DHCP?5server?5is?5not?5responding?5?$CB?$CB@ 00014f68     eboot:ebsimp.obj
 0001:00003f98       ??_C@_0BL@PFCEMBID@Error?5On?5InitDHCP?$CI?$CJ?5Call?$AN?6?$AA@ 00014f98     eboot:ebsimp.obj
 0001:00003fb4       ??_C@_0DG@KEGBCNMH@Some?5other?5station?5has?5IP?5Addres@ 00014fb4     eboot:ebsimp.obj
 0001:00003fec       ??_C@_0DA@PMFFKPM@Got?5Response?5from?5DHCP?5server?0?5I@ 00014fec     eboot:ebsimp.obj
 0001:0000401c       ??_C@_0CB@PCBFMPDH@?9EbootSendBootmeAndWaitForTftp?$AN?6@ 0001501c     eboot:ebsimp.obj
 0001:00004040       ??_C@_0CB@EEDKKNBN@?$CLEbootSendBootmeAndWaitForTftp?$AN?6@ 00015040     eboot:ebsimp.obj
 0001:00004064       ??_C@_0DF@HGBBKEBE@WARNING?3?5Some?5other?5station?5has?5@ 00015064     eboot:ebsimp.obj
 0001:0000409c       ??_C@_08NMEDJLNE@boot?4bin?$AA@ 0001509c     eboot:ebsimp.obj
 0001:000040a8       ??_C@_0CP@POPAOFAN@An?5OACK?5packet?5is?5the?5proper?5ack@ 000150a8     eboot:tftpd.obj
 0001:000040d8       ??_C@_07JPIGAOKK@blksize?$AA@ 000150d8     eboot:tftpd.obj
 0001:000040e0       ??_C@_0FD@OCECBKGJ@There?5must?5be?5an?5even?5number?0?5an@ 000150e0     eboot:tftpd.obj
 0001:00004134       ??_C@_0DB@LKOCKFPL@Illegal?5TFTP?5Operation?5?9?5Read?1Wr@ 00015134     eboot:tftpd.obj
 0001:00004168       ??_C@_0CN@LGCIOIPF@There?5were?5no?5options?5detected?5i@ 00015168     eboot:tftpd.obj
 0001:00004198       ??_C@_0FJ@NDFKPFHG@Illegal?5TFTP?5Option?5?9?5An?5option?5@ 00015198     eboot:tftpd.obj
 0001:000041f4       ??_C@_06CECHPPMB@?5?$CFd?4?$AN?6?$AA@ 000151f4     eboot:tftpd.obj
 0001:000041fc       ??_C@_0DO@FNNPCMEI@with?5a?5value?5that?5is?5out?5of?5rang@ 000151fc     eboot:tftpd.obj
 0001:0000423c       ??_C@_0DM@IIELHHA@with?5a?5value?5that?5is?5in?5range?4?$AN?6@ 0001523c     eboot:tftpd.obj
 0001:00004278       ??_C@_0BL@FNDCPDJI@The?5option?8s?5value?5is?5?$CFs?$AN?6?$AA@ 00015278     eboot:tftpd.obj
 0001:00004294       ??_C@_0CI@KEAAKLLA@This?5TFTP?5packet?5contains?5?$CFd?5opt@ 00015294     eboot:tftpd.obj
 0001:000042c0       ??_C@_0ED@FMPMEGBG@We?5currently?5only?5look?5at?5the?5fi@ 000152c0     eboot:tftpd.obj
 0001:00004304       ??_C@_0CC@KHJDBEOG@The?5packet?8s?5option?5name?5is?5?$CFs?4?$AN@ 00015304     eboot:tftpd.obj
 0001:00004328       ??_C@_0CG@JBBJIFDI@You?5must?5access?5files?5in?5binary?5@ 00015328     eboot:tftpd.obj
 0001:00004350       ??_C@_05IIBPGMLM@octet?$AA@ 00015350     eboot:tftpd.obj
 0001:00004358       ??_C@_0BG@GIKNIKEH@Locked?5Down?5Link?5?$CFd?$AN?6?$AA@ 00015358     eboot:tftpd.obj
 0001:00004370       ??_C@_0BF@JDGNCBEC@Src?5IP?5?$CFs?5Port?5?$CFH?5?5?5?$AA@ 00015370     eboot:tftpd.obj
 0001:00004388       ??_C@_0BF@MOPBEBEN@Dest?5IP?5?$CFs?5Port?5?$CFH?$AN?6?$AA@ 00015388     eboot:tftpd.obj
 0001:000043a0       ??_C@_0CL@HCAEOMAE@Default?5TFTP?5block?5size?5set?5to?3?5@ 000153a0     eboot:tftpd.obj
 0001:000043cc       ??_C@_0DB@OCKCBBAL@No?5Server?5Process?5Associated?5Wit@ 000153cc     eboot:tftpd.obj
 0001:00004400       ??_C@_0CN@CMBNFGFO@TFTP?5packet?5could?5have?5?$CFd?5name?1v@ 00015400     eboot:tftpd.obj
 0001:00004430       ??_C@_06CBLHAGFD@?$FLNULL?$FN?$AA@ 00015430     eboot:tftpd.obj
 0001:00004438       ??_C@_02HAOIJKIC@?$CFc?$AA@ 00015438     eboot:tftpd.obj
 0001:0000443c       ??_C@_0CD@NDCILIIJ@Packet?5has?5the?5following?5data?3?$AN?6@ 0001543c     eboot:tftpd.obj
 0001:00004460       ??_C@_0DJ@MEFFBBAC@TFTP?3?5Desktop?5losing?5ACK?0?5block?5@ 00015460     eboot:tftp.obj
 0001:0000449c       ??_C@_0DC@MHCCPLAO@TFtpStateMachine?3?3TFTP_STATE_CLO@ 0001549c     eboot:tftp.obj
 0001:000044d0       ??_C@_0CI@FJCIJAAP@TFTP?5Error?5Received?5From?5Host?5?$CFX@ 000154d0     eboot:tftp.obj
 0001:000044f8       ??_C@_0CG@OFKOPMJ@TftpReceiver?0?5port?3?50x?$CFX?0?5wkp?3?50@ 000154f8     eboot:tftp.obj
 0001:00004520       ??_C@_0EB@BKDEILKN@TFTP?5link?$FL?$CFu?$FN?3?5State?3?$CFu?0?5DestAdd@ 00015520     eboot:tftp.obj
 0001:00004568       ??_C@_0IO@FOKDOCNJ@Duplicate?5IP?5Address?5Detected?3?$AN?6@ 00015568     eboot:udp.obj
 0001:000045f8       ??_C@_0CJ@ICDDJIPJ@?$CBCheckUDP?3?5UDP?5header?5checksum?5f@ 000155f8     eboot:udp.obj
 0001:00004624       ??_C@_0CI@JJAKDMIL@?$CBCheckUDP?3?5IP?5header?5checksum?5fa@ 00015624     eboot:udp.obj
 0001:0000464c       ??_C@_0CE@JJEEIBJP@?$CBCheckUDP?3?5Not?5UDP?5?$CIproto?5?$DN?50x?$CFX@ 0001564c     eboot:udp.obj
 0001:00004670       ??_C@_0O@DFHLFDCO@netmask?3?5?$CFs?$AN?6?$AA@ 00015670     eboot:dhcp.obj
 0001:00004680       ??_C@_0DK@EEIOPNMG@ProcessDHCP?$CI?$CJ?3?3DHCP_INIT?3?3SendDH@ 00015680     eboot:dhcp.obj
 0001:000046bc       ??_C@_0BL@LBDFFECM@ProcessDHCP?$CI?$CJ?3?3DHCP_INIT?$AN?6?$AA@ 000156bc     eboot:dhcp.obj
 0001:000046d8       ??_C@_0DC@EKKEKBDC@ProcessDHCP?$CI?$CJ?3?3DHCP_SELECTING?3?3S@ 000156d8     eboot:dhcp.obj
 0001:00004710       ??_C@_0FK@JNLIFC@ProcessDHCP?$CI?$CJ?3?3DHCP_SELECTING?3?3D@ 00015710     eboot:dhcp.obj
 0001:00004770       ??_C@_0FI@KEBKGIEO@ProcessDHCP?$CI?$CJ?3?3DHCP_SELECTING?3?3D@ 00015770     eboot:dhcp.obj
 0001:000047c8       ??_C@_0DC@KHEOJACB@?$AN?6ProcessDHCP?$CI?$CJ?3?3DHCP?5IP?5Address@ 000157c8     eboot:dhcp.obj
 0001:000047fc       ??_C@_0BJ@MEOPKMJJ@Lease?5time?3?5?$CFd?5seconds?$AN?6?$AA@ 000157fc     eboot:dhcp.obj
 0001:00004818       ??_C@_0FI@EHEELHEE@ProcessDHCP?$CI?$CJ?3?3DHCP_REQUESTING?3?3@ 00015818     eboot:dhcp.obj
 0001:00004870       ??_C@_0DE@BHBNDGEJ@ProcessDHCP?$CI?$CJ?5Error?5?9?5No?5DHCP?5Me@ 00015870     eboot:dhcp.obj
 0001:000048a4       ??_C@_0DO@EHKMGFMI@InitDHCP?$CI?$CJ?5Error?5?9?5First?5DHCP?5Op@ 000158a4     eboot:dhcp.obj
 0001:000048e4       ??_C@_0CF@NLOHFKBD@InitDHCP?$CI?$CJ?3?3?5Calling?5ProcessDHCP@ 000158e4     eboot:dhcp.obj
 0001:0000490c       ??_C@_0DB@JKAMMNCP@EbootDHCPRetransmit?$CI?$CJ?3?3Error?5On?5@ 0001590c     eboot:dhcp.obj
 0001:00004940       ??_C@_0CN@GEBEIIOD@SendDHCP?$CI?$CJ?3?3Error?5On?5DHCPRetrans@ 00015940     eboot:dhcp.obj
 0001:00004970       ??_C@_0CG@GEIANEBC@SendDHCP?$CI?$CJ?3?3Error?5On?5SendUDP?$CI?$CJ?5C@ 00015970     eboot:dhcp.obj
 0001:00004998       ??_C@_0BD@GIINPDL@Error?5in?5SendUDP?$AN?6?$AA@ 00015998     eboot:edbg.obj
 0001:000049ac       ??_C@_0CC@IFLECHKJ@Got?5EDBG_CMD_CONFIG?0?5flags?30x?$CFX?$AN@ 000159ac     eboot:edbg.obj
 0001:000049d0       ??_C@_0BH@EBGODALL@Got?5EDBG_CMD_JUMPIMG?$AN?6?$AA@ 000159d0     eboot:edbg.obj
 0001:000049e8       ??_C@_0EE@BGOJJHDN@TFTP?5download?5started?5previously@ 000159e8     eboot:edbg.obj
 0001:00004a2c       ??_C@_0BE@MGGELJDD@Sent?5BOOTME?5to?5?$CFs?$AN?6?$AA@ 00015a2c     eboot:edbg.obj
 0001:00004a40       ??_C@_0CI@BKOJILAL@SendBootme?$CI?$CJ?3?3Error?5on?5SendUDP?$CI?$CJ@ 00015a40     eboot:edbg.obj
 0001:00004a68       pTOC                       00015a68     oal_blcommon:blcommon.obj
 0001:00004a70       NKSignon                   00015a70     oal_blcommon:blcommon.obj
 0001:00004acc       ??_C@_0DJ@LFHEGALA@ERROR?3?5Checksum?5failure?5?$CIexpecte@ 00015acc     oal_blcommon:blcommon.obj
 0001:00004b08       ??_C@_0BM@DKIOIAMD@?$AN?6BL_IMAGE_TYPE_UNKNOWN?$AN?6?$AN?6?$AA@ 00015b08     oal_blcommon:blcommon.obj
 0001:00004b24       ??_C@_0BP@KNNCEABF@?$AN?6BL_IMAGE_TYPE_SIGNED_NB0?$AN?6?$AN?6?$AA@ 00015b24     oal_blcommon:blcommon.obj
 0001:00004b44       ??_C@_07LAGBNAEN@R000FF?6?$AA@ 00015b44     oal_blcommon:blcommon.obj
 0001:00004b4c       ??_C@_0BP@MJFCGNBB@?$AN?6BL_IMAGE_TYPE_SIGNED_BIN?$AN?6?$AN?6?$AA@ 00015b4c     oal_blcommon:blcommon.obj
 0001:00004b6c       ??_C@_07HMMLNAND@S000FF?6?$AA@ 00015b6c     oal_blcommon:blcommon.obj
 0001:00004b74       ??_C@_0BI@HBMHAEFD@?$AN?6BL_IMAGE_TYPE_BIN?$AN?6?$AN?6?$AA@ 00015b74     oal_blcommon:blcommon.obj
 0001:00004b8c       ??_C@_07MMNKOBGG@B000FF?6?$AA@ 00015b8c     oal_blcommon:blcommon.obj
 0001:00004b94       ??_C@_0BN@IHLEHBEK@?$AN?6BL_IMAGE_TYPE_MULTIXIP?$AN?6?$AN?6?$AA@ 00015b94     oal_blcommon:blcommon.obj
 0001:00004bb4       ??_C@_07CBKBMMIF@X000FF?6?$AA@ 00015bb4     oal_blcommon:blcommon.obj
 0001:00004bbc       ??_C@_0BN@GCKOHOON@?$AN?6BL_IMAGE_TYPE_MANIFEST?$AN?6?$AN?6?$AA@ 00015bbc     oal_blcommon:blcommon.obj
 0001:00004bdc       ??_C@_07JLHFPECJ@N000FF?6?$AA@ 00015bdc     oal_blcommon:blcommon.obj
 0001:00004be4       ??_C@_0CL@OKMIEAHJ@?$AN?6ERROR?3?5Unable?5to?5read?5image?5si@ 00015be4     oal_blcommon:blcommon.obj
 0001:00004c10       ??_C@_0DJ@PIPLIHFI@?$AN?6ERROR?3?5Unable?5to?5read?5download@ 00015c10     oal_blcommon:blcommon.obj
 0001:00004c50       ??_C@_0EC@LAKEOKID@?$AN?6ERROR?3?5Download?5manifest?5packe@ 00015c50     oal_blcommon:blcommon.obj
 0001:00004c94       ??_C@_0DG@DBBGHEAG@?$AN?6ERROR?3?5Unable?5to?5read?5download@ 00015c94     oal_blcommon:blcommon.obj
 0001:00004ccc       ??_C@_0DL@DCHMDHHD@ImageStart?5?$DN?50x?$CFx?0?5ImageLength?5?$DN@ 00015ccc     oal_blcommon:blcommon.obj
 0001:00004d08       ??_C@_0CO@PFLGIDFG@ERROR?3?5failed?5when?5reading?5raw?5b@ 00015d08     oal_blcommon:blcommon.obj
 0001:00004d38       ??_C@_0BP@EOFEMPOO@Invalid?5flash?5address?1length?$AN?6?$AA@ 00015d38     oal_blcommon:blcommon.obj
 0001:00004d58       ??_C@_0CC@DNECAMLM@?$CBOEMVERIFYMEMORY?3?5Invalid?5image?$AN@ 00015d58     oal_blcommon:blcommon.obj
 0001:00004d7c       ??_C@_0DH@GJCJAHAP@?$FL?$CFd?$FN?3?5Address?$DN0x?$CFx?5?5Length?$DN0x?$CFx?5@ 00015d7c     oal_blcommon:blcommon.obj
 0001:00004db4       ??_C@_03ILDADBHF@RAM?$AA@  00015db4     oal_blcommon:blcommon.obj
 0001:00004db8       ??_C@_05HPMNGINJ@FLASH?$AA@ 00015db8     oal_blcommon:blcommon.obj
 0001:00004dc0       ??_C@_0BH@FIOKDOBJ@?$AN?6Completed?5file?$CIs?$CJ?3?$AN?6?$AA@ 00015dc0     oal_blcommon:blcommon.obj
 0001:00004dd8       ??_C@_0FC@PGPOMBFM@?9?9?9?9?9?9?9?9?9?9?9?9?9?9?9?9?9?9?9?9?9?9?9?9?9?9?9?9?9?9?9?9@ 00015dd8     oal_blcommon:blcommon.obj
 0001:00004e2c       ??_C@_06OLEINIPO@nk?4exe?$AA@ 00015e2c     oal_blcommon:blcommon.obj
 0001:00004e34       ??_C@_0CE@NKAMCDHO@Unable?5to?5read?5image?5start?1lengt@ 00015e34     oal_blcommon:blcommon.obj
 0001:00004e58       ??_C@_0DI@FDIIHFBA@?$CK?$CK?$CK?$CK?$CK?$CK?5Checksum?5failure?5on?5recor@ 00015e58     oal_blcommon:blcommon.obj
 0001:00004e90       ??_C@_0DD@KHJBCIED@?$CK?$CK?$CK?$CK?$CK?$CK?5Data?5record?5?$CFd?5corrupted?0@ 00015e90     oal_blcommon:blcommon.obj
 0001:00004ec4       ??_C@_0BD@PHLGNLDI@rom_offset?$DN0x?$CFx?4?$AN?6?$AA@ 00015ec4     oal_blcommon:blcommon.obj
 0001:00004ed8       ??_C@_0EC@NABDPCJO@?$CK?$CK?5ERROR?3?5This?5boot?5loader?5does?5@ 00015ed8     oal_blcommon:blcommon.obj
 0001:00004f20       ??_C@_0EC@MIGFFFAC@?$CK?$CK?5ERROR?3?5This?5boot?5loader?5does?5@ 00015f20     oal_blcommon:blcommon.obj
 0001:00004f64       ??_C@_06BEBGGBAB@?$AN?6?$CK?$CK?$AN?6?$AA@ 00015f64     oal_blcommon:blcommon.obj
 0001:00004f70       ??_C@_0GI@NIAHKKOO@?$CK?$CK?5ERROR?3?5The?5X000FF?5packet?5is?5a@ 00015f70     oal_blcommon:blcommon.obj
 0001:00004fd8       ??_C@_0FO@KDFAPMNM@?$CK?$CK?5Please?5update?5your?5Platform?5B@ 00015fd8     oal_blcommon:blcommon.obj
 0001:00005038       ??_C@_04IPBEALME@?$CK?$CK?$AN?6?$AA@ 00016038     oal_blcommon:blcommon.obj
 0001:00005040       ??_C@_0BI@OCFAEGPK@ROMHDR?5at?5Address?5?$CFXh?$AN?6?$AA@ 00016040     oal_blcommon:blcommon.obj
 0001:00005058       ??_C@_0CL@NOFKHKJC@System?5ready?$CB?$AN?6Preparing?5for?5dow@ 00016058     oal_blcommon:blcommon.obj
 0001:00005084       ??_C@_1BI@FCMLLAGN@?$AA?$CF?$AAd?$AA?4?$AA?$CF?$AAd?$AA?4?$AA?$CF?$AAd?$AA?4?$AA?$CF?$AAd?$AA?$AA@ 00016084     oal_kitl:format.obj
 0001:0000509c       ??_C@_1DM@BKFFFBIH@?$AA?$CF?$AA0?$AA2?$AAx?$AA?3?$AA?$CF?$AA0?$AA2?$AAx?$AA?3?$AA?$CF?$AA0?$AA2?$AAx?$AA?3?$AA?$CF?$AA0?$AA2?$AAx?$AA?3?$AA?$CF?$AA0?$AA2?$AAx?$AA?3?$AA?$CF?$AA0?$AA2?$AAx?$AA?$AA@ 0001609c     oal_kitl:format.obj
 0001:000050d8       ??_C@_0EH@LPLMFKIL@?$AN?6?9?9?9?9?9?9?9?9?9?9?9?9?9?9?9?9?9?9?9?9?9?9?9?9?9?9?9?9?9?5@ 000160d8     bootshell_common_topaz_v1:bootshell.obj
 0001:00005120       ??_C@_0DJ@JLNEADMA@?$DP?5?5?5?5?5?5?5?5?5?5?5?5?5?5?5?5?5?5?5?5?5?5?5?5?5?5?5?5?5?5?5@ 00016120     bootshell_common_topaz_v1:bootshell.obj
 0001:0000515c       ??_C@_0DP@MKCEOKDD@e?5?5?5?5?5?5?5?5?5?5?5?5?5?5?5?5?5?5?5?5?5?5?5?5?5?5?5?5?5?5?5@ 0001615c     bootshell_common_topaz_v1:bootshell.obj
 0001:0000519c       ??_C@_0DN@NGLAIDIN@d?5RegAddress?5?5?5?5?5?5?5?5?5?5?5?5?5?5?5?5?5?5?5?5@ 0001619c     bootshell_common_topaz_v1:bootshell.obj
 0001:000051dc       ??_C@_0DM@OGKFCBKC@s?5RegAddress?5RegValue?5?5?5?5?5?5?5?5?5?5?5@ 000161dc     bootshell_common_topaz_v1:bootshell.obj
 0001:00005218       ??_C@_0DM@EAFILELA@b?5RegAddress?5BitOffset?$CI0?931?$CJ?5Val@ 00016218     bootshell_common_topaz_v1:bootshell.obj
 0001:00005258       ??_C@_0EG@IMDNCDIO@?9?9?9?9?9?9?9?9?9?9?9?9?9?9?9?9?9?9?9?9?9?9?9?9?9?9?9?9?9?9?5E@ 00016258     bootshell_common_topaz_v1:bootshell.obj
 0001:000052a0       ??_C@_0DJ@BIKMIJAN@?$AN?6All?5the?5input?5parameters?5are?5s@ 000162a0     bootshell_common_topaz_v1:bootshell.obj
 0001:000052dc       ??_C@_0CM@CFBEBIAI@New?5Info?5?3?5?5Reg?5Addr?5?$DN?50x?$CFx?0Valu@ 000162dc     bootshell_common_topaz_v1:bootshell.obj
 0001:00005308       ??_C@_0CH@NHPNKMID@Invalid?5Address?0Please?5Input?5Aga@ 00016308     bootshell_common_topaz_v1:bootshell.obj
 0001:00005330       ??_C@_0CH@PFJMOMPP@Physical?5Reg?5Addr?5?$DN?5?$CFs?0Value?5?$DN?50@ 00016330     bootshell_common_topaz_v1:bootshell.obj
 0001:00005358       ??_C@_0CJ@JNGMHGML@Invalid?5Bit?5index?0Please?5Input?5A@ 00016358     bootshell_common_topaz_v1:bootshell.obj
 0001:00005384       ??_C@_0CL@FFJBHPMN@New?5Info?5?3?5Reg?5Addr?5?$DN?50x?$CFx?0Value@ 00016384     bootshell_common_topaz_v1:bootshell.obj
 0001:000053e0       OEMBootInit                000163e0 f   eboot.obj
 0001:00005418       OEMGetMagicNumber          00016418 f   eboot.obj
 0001:00005424       GetPreDownloadInfo         00016424 f   eboot.obj
 0001:0000557c       GetLaunchInfo              0001657c f   eboot.obj
 0001:000056b8       OEMReadData                000166b8 f   eboot.obj
 0001:000056e0       ResetDefaultBootCFG        000166e0 f   eboot.obj
 0001:000057c8       OEMEthGetFrame             000167c8 f   eboot.obj
 0001:000057e8       OEMEthSendFrame            000167e8 f   eboot.obj
 0001:00005a4c       BLMenu                     00016a4c f   menu.obj
 0001:00005d5c       KITLOutputDebugString      00016d5c f   oal_blnk:wrappersa.obj
 0001:00005da8       NKsprintfA                 00016da8 f   oal_blnk:wrappersa.obj
 0001:00005dd0       inet_ntoa                  00016dd0 f   oal_blnk:ipformata.obj
 0001:00005e24       inet_addr                  00016e24 f   oal_blnk:ipformata.obj
 0001:00005e80       NKvsprintfA                00016e80 f   oal_blnk:formata.obj
 0001:00006820       OALPAtoVA                  00017820 f   oal_blmemory_arm:memory.obj
 0001:00006898       OALVAtoPA                  00017898 f   oal_blmemory_arm:memory.obj
 0001:00006918       OALSerialInit              00017918 f   bspcmn:debugserial.obj
 0001:00006954       OEMInitDebugSerial         00017954 f   bspcmn:debugserial.obj
 0001:00006a9c       OEMWriteDebugByte          00017a9c f   bspcmn:debugserial.obj
 0001:00006ac8       OEMReadDebugByte           00017ac8 f   bspcmn:debugserial.obj
 0001:00006af0       OEMWriteDebugLED           00017af0 f   bspcmn:debugserial.obj
 0001:00006af4       OALBspArgsInit             00017af4 f   bspcmn:bspargs.obj
 0001:00006f08       OALBspArgsPrint            00017f08 f   bspcmn:bspargs.obj
 0001:00006f0c       main                       00017f0c f   bootcmn:main.obj
 0001:00006f28       OEMDebugInit               00017f28 f   bootcmn:main.obj
 0001:00006f38       OEMPreDownload             00017f38 f   bootcmn:main.obj
 0001:000070c0       OEMLaunch                  000180c0 f   bootcmn:main.obj
 0001:00007188       OEMMultiBINNotify          00018188 f   bootcmn:main.obj
 0001:000074d4       OEMReportError             000184d4 f   bootcmn:main.obj
 0001:000074f0       OEMVerifyMemory            000184f0 f   bootcmn:main.obj
 0001:00007790       StoreBootCFG               00018790 f   bootcmn:main.obj
 0001:000077c0       LoadBootCFG                000187c0 f   bootcmn:main.obj
 0001:00007834       ConfigBootCFG              00018834 f   bootcmn:main.obj
 0001:000078b0       OEMPlatformInit            000188b0 f   bootcmn:main.obj
 0001:00007c68       InitSpecifiedEthDevice     00018c68 f   bootcmn:ether.obj
 0001:00007e44       OEMReset                   00018e44 f   bootcmn:utils.obj
 0001:00007e70       SpinForever                00018e70 f   bootcmn:utils.obj
 0001:00007ea8       OEMShowProgress            00018ea8 f   bootcmn:utils.obj
 0001:00007eac       BootTimerInit              00018eac f   bootcmn:utils.obj
 0001:00007f00       OALClockSetGatingMode      00018f00 f   bootcmn:utils.obj
 0001:00007f48       SetDelay                   00018f48 f   bootcmn:utils.obj
 0001:00008040       NKCreateStaticMapping      00019040 f   bootcmn:utils.obj
 0001:0000804c       OEMIsFlashAddr             0001904c f   bootcmn:flash.obj
 0001:00008080       OEMMapMemAddr              00019080 f   bootcmn:flash.obj
 0001:0000810c       OEMStartEraseFlash         0001910c f   bootcmn:flash.obj
 0001:00008144       OEMContinueEraseFlash      00019144 f   bootcmn:flash.obj
 0001:00008184       OEMFinishEraseFlash        00019184 f   bootcmn:flash.obj
 0001:000081b4       OEMWriteFlash              000191b4 f   bootcmn:flash.obj
 0001:000083a8       FlashLoadBootCFG           000193a8 f   bootcmn:flash.obj
 0001:00008408       FlashStoreBootCFG          00019408 f   bootcmn:flash.obj
 0001:00008468       SPIWriteXldr               00019468 f   bootcmn:cspi_flash.obj
 0001:000085bc       SPIWriteBoot               000195bc f   bootcmn:cspi_flash.obj
 0001:00008850       SPILoadBootCFG             00019850 f   bootcmn:cspi_flash.obj
 0001:00008954       SPIStoreBootCFG            00019954 f   bootcmn:cspi_flash.obj
 0001:00008ac0       PageWrite                  00019ac0 f   bootcmn:i2c_eeprom.obj
 0001:00008b8c       PageRead                   00019b8c f   bootcmn:i2c_eeprom.obj
 0001:00008c74       IsWriteOperationComplete   00019c74 f   bootcmn:i2c_eeprom.obj
 0001:00008cf4       I2CEEPROMWriteXldr         00019cf4 f   bootcmn:i2c_eeprom.obj
 0001:00008e18       OALConfigSerialUART        00019e18 f   serialutils:serialutils.obj
 0001:00008fd8       OALConfigSerialIOMUX       00019fd8 f   serialutils:serialutils.obj
 0001:00009044       OALStall                   0001a044 f   ethdrv:ethdrv.obj
 0001:00009180       OEMKitlGetSecs             0001a180 f   ethdrv:ethdrv.obj
 0001:00009264       OEMEthGetSecs              0001a264 f   ethdrv:ethdrv.obj
 0001:00009268       BLMenuEnableDisable        0001a268 f   blmenu_common_topaz_v1:menu.obj
 0001:000092b0       BLMenuReadLine             0001a2b0 f   blmenu_common_topaz_v1:menu.obj
 0001:00009364       BLMenuPrintData            0001a364 f   blmenu_common_topaz_v1:menu.obj
 0001:0000959c       BLMenuBootShell            0001a59c f   blmenu_common_topaz_v1:menu.obj
 0001:000095ac       BLMenuSaveSettings         0001a5ac f   blmenu_common_topaz_v1:menu.obj
 0001:000095dc       BLMenuReset                0001a5dc f   blmenu_common_topaz_v1:menu.obj
 0001:000095ec       BLMenuLaunchFlashImage     0001a5ec f   blmenu_common_topaz_v1:menu.obj
 0001:00009604       BLMenuBootDelay            0001a604 f   blmenu_common_topaz_v1:menu.obj
 0001:00009628       BLMenuResetConfiguration   0001a628 f   blmenu_common_topaz_v1:menu.obj
 0001:0000963c       BLMenuDownloadImageNow     0001a63c f   blmenu_common_topaz_v1:menu.obj
 0001:00009654       BLMenuFormatNandOS         0001a654 f   blmenu_common_topaz_v1:menu.obj
 0001:000096a8       BLMenuFormatAllNand        0001a6a8 f   blmenu_common_topaz_v1:menu.obj
 0001:00009708       BLMenuEMMCToggleBP         0001a708 f   blmenu_common_topaz_v1:menu.obj
 0001:00009728       BLMenuEMMCBPSize           0001a728 f   blmenu_common_topaz_v1:menu.obj
 0001:0000979c       BLMenuESDBPEnable          0001a79c f   blmenu_common_topaz_v1:menu.obj
 0001:000097ac       BLMenuESDBPSize            0001a7ac f   blmenu_common_topaz_v1:menu.obj
 0001:00009820       BLMenuFormatAllSDMMC       0001a820 f   blmenu_common_topaz_v1:menu.obj
 0001:00009880       BLMenuCreateFileSystemOnSDMMC 0001a880 f   blmenu_common_topaz_v1:menu.obj
 0001:00009900       BLMenuReturn               0001a900 f   blmenu_common_topaz_v1:menu.obj
 0001:00009908       BLMenuShow                 0001a908 f   blmenu_common_topaz_v1:menu.obj
 0001:00009ae8       BLMenuSetMacAddress        0001aae8 f   blmenu_common_topaz_v1:menu.obj
 0001:00009be8       BLMenuSetIpAddress         0001abe8 f   blmenu_common_topaz_v1:menu.obj
 0001:00009cb8       BLMenuSetIpMask            0001acb8 f   blmenu_common_topaz_v1:menu.obj
 0001:00009d80       BLMenuMMCSDUtilities       0001ad80 f   blmenu_common_topaz_v1:menu.obj
 0001:00009f88       BspBootShell               0001af88 f   bsp_bootshell:bspbootshell.obj
 0001:0000a18c       MIIREAD                    0001b18c f   oal_ethdrv_fec_common_topaz_v1:fec.obj
 0001:0000a218       MIIWRITE                   0001b218 f   oal_ethdrv_fec_common_topaz_v1:fec.obj
 0001:0000a26c       FECEnableInts              0001b26c f   oal_ethdrv_fec_common_topaz_v1:fec.obj
 0001:0000a284       FECDisableInts             0001b284 f   oal_ethdrv_fec_common_topaz_v1:fec.obj
 0001:0000a29c       FECInitDMABuffer           0001b29c f   oal_ethdrv_fec_common_topaz_v1:fec.obj
 0001:0000a424       FECInit                    0001b424 f   oal_ethdrv_fec_common_topaz_v1:fec.obj
 0001:0000a834       FECSendFrame               0001b834 f   oal_ethdrv_fec_common_topaz_v1:fec.obj
 0001:0000a910       FECGetFrame                0001b910 f   oal_ethdrv_fec_common_topaz_v1:fec.obj
 0001:0000aa4c       OALKitlFECBSPInit          0001ba4c f   bspfec:bspfec.obj
 0001:0000abc4       BSPFECusesRMII             0001bbc4 f   bspfec:bspfec.obj
 0001:0000abcc       RndisRestart               0001bbcc f   fsl_rne_mdd_common_topaz_v1:rndis.obj
 0001:0000ac2c       RndisPrepareRndisPacket    0001bc2c f   fsl_rne_mdd_common_topaz_v1:rndis.obj
 0001:0000accc       MddSendRndisPacketComplete 0001bccc f   fsl_rne_mdd_common_topaz_v1:rndis.obj
 0001:0000ace0       RndisEDbgSendFrame         0001bce0 f   fsl_rne_mdd_common_topaz_v1:rndis.obj
 0001:0000ae10       MddSendRndisMessageComplete 0001be10 f   fsl_rne_mdd_common_topaz_v1:rndis.obj
 0001:0000ae38       RndisSendRndisMessage      0001be38 f   fsl_rne_mdd_common_topaz_v1:rndis.obj
 0001:0000b04c       RndisProcessMessage        0001c04c f   fsl_rne_mdd_common_topaz_v1:rndis.obj
 0001:0000b3f8       RndisEDbgGetFrame          0001c3f8 f   fsl_rne_mdd_common_topaz_v1:rndis.obj
 0001:0000b544       RndisProcessPacket         0001c544 f   fsl_rne_mdd_common_topaz_v1:rndis.obj
 0001:0000b684       RndisInit                  0001c684 f   fsl_rne_mdd_common_topaz_v1:rndis.obj
 0001:0000b894       RndisEnableInts            0001c894 f   fsl_rne_mdd_common_topaz_v1:rndis.obj
 0001:0000b8b8       RndisDisableInts           0001c8b8 f   fsl_rne_mdd_common_topaz_v1:rndis.obj
 0001:0000b8dc       HostMiniQueryInformation   0001c8dc f   fsl_rne_mdd_common_topaz_v1:hostmini.obj
 0001:0000bbc0       HostMiniSetInformation     0001cbc0 f   fsl_rne_mdd_common_topaz_v1:hostmini.obj
 0001:0000bd04       MddIndicateRndisMessage    0001cd04 f   fsl_rne_mdd_common_topaz_v1:hostmini.obj
 0001:0000bd08       MddIndicateRndisPacket     0001cd08 f   fsl_rne_mdd_common_topaz_v1:hostmini.obj
 0001:0000bd24       MDDAllocDataWrapper        0001cd24 f   fsl_rne_mdd_common_topaz_v1:hostmini.obj
 0001:0000bd4c       MDDFreeMem                 0001cd4c f   fsl_rne_mdd_common_topaz_v1:hostmini.obj
 0001:0000bd50       MDDFreeDataWrapper         0001cd50 f   fsl_rne_mdd_common_topaz_v1:hostmini.obj
 0001:0000bd64       HostMiniInit               0001cd64 f   fsl_rne_mdd_common_topaz_v1:hostmini.obj
 0001:0000bda0       InitBuffer                 0001cda0 f   fsl_rne_mdd_common_topaz_v1:util.obj
 0001:0000be38       AvaiableBufferSize         0001ce38 f   fsl_rne_mdd_common_topaz_v1:util.obj
 0001:0000be74       AllocBuffer                0001ce74 f   fsl_rne_mdd_common_topaz_v1:util.obj
 0001:0000bf5c       FreeBuffer                 0001cf5c f   fsl_rne_mdd_common_topaz_v1:util.obj
 0001:0000c0dc       GetFirstUsedBuffer         0001d0dc f   fsl_rne_mdd_common_topaz_v1:util.obj
 0001:0000c1d0       PDD_GetDescriptor          0001d1d0 f   fsl_rne_pdd_common_topaz_v1:rndis_pdd.obj
 0001:0000c33c       PDD_DoVendorCommand        0001d33c f   fsl_rne_pdd_common_topaz_v1:rndis_pdd.obj
 0001:0000c464       setupDataOutTransfer       0001d464 f   fsl_rne_pdd_common_topaz_v1:rndis_pdd.obj
 0001:0000c52c       HandleSetupPacket          0001d52c f   fsl_rne_pdd_common_topaz_v1:rndis_pdd.obj
 0001:0000c824       PDD_SendRndisMessage       0001d824 f   fsl_rne_pdd_common_topaz_v1:rndis_pdd.obj
 0001:0000c8b0       PDD_SendRndisPacket        0001d8b0 f   fsl_rne_pdd_common_topaz_v1:rndis_pdd.obj
 0001:0000c960       PDD_Set                    0001d960 f   fsl_rne_pdd_common_topaz_v1:rndis_pdd.obj
 0001:0000ca48       PDD_Get                    0001da48 f   fsl_rne_pdd_common_topaz_v1:rndis_pdd.obj
 0001:0000cb18       PDD_ISR                    0001db18 f   fsl_rne_pdd_common_topaz_v1:rndis_pdd.obj
 0001:0000cb34       PDD_IndicateRndisPacketComplete 0001db34 f   fsl_rne_pdd_common_topaz_v1:rndis_pdd.obj
 0001:0000cb58       SetRNDISSerialNumber       0001db58 f   fsl_rne_pdd_common_topaz_v1:rndis_pdd.obj
 0001:0000cbf8       NotifyHandler              0001dbf8 f   fsl_rne_pdd_common_topaz_v1:rndis_pdd.obj
 0001:0000cff8       PDDInit                    0001dff8 f   fsl_rne_pdd_common_topaz_v1:rndis_pdd.obj
 0001:0000d2a8       ClearUsbstsUI              0001e2a8 f   usb_usbfn_mx25_topaz_v1:i_pdd.obj
 0001:0000da24       UfnPdd_PowerDown           0001ea24 f   usb_usbfn_mx25_topaz_v1:i_pdd.obj
 0001:0000db08       UfnPdd_PowerUp             0001eb08 f   usb_usbfn_mx25_topaz_v1:i_pdd.obj
 0001:0000dbf4       UpdateDevicePower          0001ebf4 f   usb_usbfn_mx25_topaz_v1:i_pdd.obj
 0001:0000dcac       SetupEvent                 0001ecac f   usb_usbfn_mx25_topaz_v1:i_pdd.obj
 0001:0000dde8       CopyFromUncachedBuffer     0001ede8 f   usb_usbfn_mx25_topaz_v1:i_pdd.obj
 0001:0000e1a4       UfnPdd_IssueTransfer       0001f1a4 f   usb_usbfn_mx25_topaz_v1:i_pdd.obj
 0001:0000e778       UfnPdd_AbortTransfer       0001f778 f   usb_usbfn_mx25_topaz_v1:i_pdd.obj
 0001:0000e920       UfnPdd_StallEndpoint       0001f920 f   usb_usbfn_mx25_topaz_v1:i_pdd.obj
 0001:0000e9ac       UfnPdd_ClearEndpointStall  0001f9ac f   usb_usbfn_mx25_topaz_v1:i_pdd.obj
 0001:0000ea4c       UfnPdd_IsEndpointHalted    0001fa4c f   usb_usbfn_mx25_topaz_v1:i_pdd.obj
 0001:0000eab4       UfnPdd_SendControlStatusHandshake 0001fab4 f   usb_usbfn_mx25_topaz_v1:i_pdd.obj
 0001:0000eb34       UfnPdd_InitiateRemoteWakeup 0001fb34 f   usb_usbfn_mx25_topaz_v1:i_pdd.obj
 0001:0000eb3c       SetPowerState              0001fb3c f   usb_usbfn_mx25_topaz_v1:i_pdd.obj
 0001:0000eb80       UfnPdd_IOControl           0001fb80 f   usb_usbfn_mx25_topaz_v1:i_pdd.obj
 0001:0000ed90       UfnPdd_Deinit              0001fd90 f   usb_usbfn_mx25_topaz_v1:i_pdd.obj
 0001:0000eda0       UfnPdd_DeregisterDevice    0001fda0 f   usb_usbfn_mx25_topaz_v1:i_pdd.obj
 0001:0000eda8       UfnPdd_Stop                0001fda8 f   usb_usbfn_mx25_topaz_v1:i_pdd.obj
 0001:0000ee14       UfnPdd_DeinitEndpoint      0001fe14 f   usb_usbfn_mx25_topaz_v1:i_pdd.obj
 0001:0000eeb8       UfnPdd_InitEndpoint        0001feb8 f   usb_usbfn_mx25_topaz_v1:i_pdd.obj
 0001:0000efd4       UfnPdd_SetAddress          0001ffd4 f   usb_usbfn_mx25_topaz_v1:i_pdd.obj
 0001:0000f008       UfnPdd_Start               00020008 f   usb_usbfn_mx25_topaz_v1:i_pdd.obj
 0001:0000f0f8       UfnPdd_RegisterDevice      000200f8 f   usb_usbfn_mx25_topaz_v1:i_pdd.obj
 0001:0000f324       UfnPdd_IsEndpointSupportable 00020324 f   usb_usbfn_mx25_topaz_v1:i_pdd.obj
 0001:0000f340       UfnPdd_IsConfigurationSupportable 00020340 f   usb_usbfn_mx25_topaz_v1:i_pdd.obj
 0001:0000f494       UfnPdd_Init                00020494 f   usb_usbfn_mx25_topaz_v1:i_pdd.obj
 0001:0000f790       CheckEndpoint              00020790 f   usb_usbfn_mx25_topaz_v1:i_pdd.obj
 0001:0000fc14       InterruptHandle            00020c14 f   usb_usbfn_mx25_topaz_v1:i_pdd.obj
 0001:0001020c       FslUfnGetUsbFnPdd          0002120c f   usb_usbfn_eboot_mx25_topaz_v1:i_stub.obj
 0001:00010218       FslUfnRequestIrq           00021218 f   usb_usbfn_eboot_mx25_topaz_v1:i_stub.obj
 0001:00010220       FslUfnIsUSBKitlEnable      00021220 f   usb_usbfn_eboot_mx25_topaz_v1:i_stub.obj
 0001:00010228       FslUfnCreateThread         00021228 f   usb_usbfn_eboot_mx25_topaz_v1:i_stub.obj
 0001:00010230       UsbFnInterruptThread       00021230 f   usb_usbfn_eboot_mx25_topaz_v1:i_stub.obj
 0001:00010254       FslUfnTrigIrq              00021254 f   usb_usbfn_eboot_mx25_topaz_v1:i_stub.obj
 0001:00010278       FslUfnDeinit               00021278 f   usb_usbfn_eboot_mx25_topaz_v1:i_stub.obj
 0001:0001027c       FslUfnGetDMABuffer         0002127c f   usb_usbfn_eboot_mx25_topaz_v1:i_stub.obj
 0001:000102f8       BSPUSBClockSwitch          000212f8 f   usb_usbfn_eboot_mx25_topaz_v1:i_stub.obj
 0001:00010300       BSPUSBClockCreateFileMapping 00021300 f   usb_usbfn_eboot_mx25_topaz_v1:i_stub.obj
 0001:00010308       GetDeviceRegistryParams    00021308 f   usb_usbfn_eboot_mx25_topaz_v1:i_stub.obj
 0001:00010328       SetInterruptEvent          00021328 f   usb_usbfn_eboot_mx25_topaz_v1:i_stub.obj
 0001:00010358       FslUfnGetPageNumber        00021358 f   usb_usbfn_eboot_mx25_topaz_v1:i_stub.obj
 0001:00010378       FslUfnGetPageSize          00021378 f   usb_usbfn_eboot_mx25_topaz_v1:i_stub.obj
 0001:00010380       FslUfnGetPageShift         00021380 f   usb_usbfn_eboot_mx25_topaz_v1:i_stub.obj
 0001:00010388       FslInitializeCriticalSection 00021388 f   usb_usbfn_eboot_mx25_topaz_v1:i_stub.obj
 0001:0001038c       FslEnterCriticalSection    0002138c f   usb_usbfn_eboot_mx25_topaz_v1:i_stub.obj
 0001:00010390       FslLeaveCriticalSection    00021390 f   usb_usbfn_eboot_mx25_topaz_v1:i_stub.obj
 0001:00010394       CreateBusAccessHandle      00021394 f   usb_usbfn_eboot_mx25_topaz_v1:i_stub.obj
 0001:0001039c       CeLogData                  0002139c f   usb_usbfn_eboot_mx25_topaz_v1:i_stub.obj
 0001:000103a0       MmMapIoSpace               000213a0 f   usb_usbfn_eboot_mx25_topaz_v1:i_stub.obj
 0001:000103bc       InterruptDisable           000213bc f   usb_usbfn_eboot_mx25_topaz_v1:i_stub.obj
 0001:000103c0       CacheSync                  000213c0 f   usb_usbfn_eboot_mx25_topaz_v1:i_stub.obj
 0001:000103d0       LockPages                  000213d0 f   usb_usbfn_eboot_mx25_topaz_v1:i_stub.obj
 0001:000103e8       GetLastError               000213e8 f   usb_usbfn_eboot_mx25_topaz_v1:i_stub.obj
 0001:000103f0       UnlockPages                000213f0 f   usb_usbfn_eboot_mx25_topaz_v1:i_stub.obj
 0001:000103f8       CeOpenCallerBuffer         000213f8 f   usb_usbfn_eboot_mx25_topaz_v1:i_stub.obj
 0001:00010404       CeCloseCallerBuffer        00021404 f   usb_usbfn_eboot_mx25_topaz_v1:i_stub.obj
 0001:0001040c       StringCchLengthW           0002140c f   usb_usbfn_eboot_mx25_topaz_v1:i_stub.obj
 0001:00010420       StringCchVPrintfW          00021420 f   usb_usbfn_eboot_mx25_topaz_v1:i_stub.obj
 0001:00010428       SetDevicePowerState        00021428 f   usb_usbfn_eboot_mx25_topaz_v1:i_stub.obj
 0001:00010430       Sleep                      00021430 f   usb_usbfn_eboot_mx25_topaz_v1:i_stub.obj
 0001:00010434       CacheRangeFlush            00021434 f   usb_usbfn_eboot_mx25_topaz_v1:i_stub.obj
 0001:00010494       ?CalcChksum@@YAEPAEG@Z     00021494 f   oal_blserial:serfuncs.obj
 0001:000104e0       SerialSendBootRequest      000214e0 f   oal_blserial:serfuncs.obj
 0001:000105a0       SerialSendBlockAck         000215a0 f   oal_blserial:serfuncs.obj
 0001:00010640       RecvHeader                 00021640 f   oal_blserial:serfuncs.obj
 0001:00010720       RecvPacket                 00021720 f   oal_blserial:serfuncs.obj
 0001:00010820       SerialReadData             00021820 f   oal_blserial:serfuncs.obj
 0001:000109c0       SerialWaitForBootAck       000219c0 f   oal_blserial:serfuncs.obj
 0001:00010a74       SerialWaitForJump          00021a74 f   oal_blserial:serfuncs.obj
 0001:00010de0       ?HandleGetDescriptor@@YAXPAU_USB_DEVICE_REQUEST@@PAU_EP0_REQUEST@@@Z 00021de0 f   fsl_serial_pdd_common_topaz_v1:serial_dl.obj
 0001:00010e6c       ?HandleTransferComplete@@YAXPAU_STransfer@@@Z 00021e6c f   fsl_serial_pdd_common_topaz_v1:serial_dl.obj
 0001:00011208       USBSerialInit              00022208 f   fsl_serial_pdd_common_topaz_v1:serial_dl.obj
 0001:000112e4       OEMSerialSendRaw           000222e4 f   fsl_serial_pdd_common_topaz_v1:serial_dl.obj
 0001:000113cc       OEMSerialRecvRaw           000223cc f   fsl_serial_pdd_common_topaz_v1:serial_dl.obj
 0001:00011598       GetRNDISMACAddress         00022598 f   fsl_usbfn_rndiskitl_mx25_topaz_v1:hwinit.obj
 0001:000115c8       controllerSetup            000225c8 f   fsl_usbfn_rndiskitl_mx25_topaz_v1:hwinit.obj
 0001:00011680       HardwareInitialize         00022680 f   fsl_usbfn_rndiskitl_mx25_topaz_v1:hwinit.obj
 0001:0001174c       PowerDownSchemeExist       0002274c f   fsl_usbfn_rndiskitl_mx25_topaz_v1:hwinit.obj
 0001:00011754       BSPUsbXvrEnableVBUSIntr    00022754 f   fsl_usbfn_rndiskitl_mx25_topaz_v1:hwinit.obj
 0001:00011770       BSPUsbResetPHY             00022770 f   fsl_usbfn_rndiskitl_mx25_topaz_v1:hwinit.obj
 0001:00011774       BSPUsbSetBusConfig         00022774 f   fsl_usbfn_rndiskitl_mx25_topaz_v1:hwinit.obj
 0001:00011784       BSPUSBInterruptControl     00022784 f   fsl_usbfn_rndiskitl_mx25_topaz_v1:hwinit.obj
 0001:00011788       BSPPhyShowDevDiscon        00022788 f   fsl_usbfn_rndiskitl_mx25_topaz_v1:hwinit.obj
 0001:00011790       BSPUsbSetCurrentLimitation 00022790 f   fsl_usbfn_rndiskitl_mx25_topaz_v1:hwinit.obj
 0001:00011794       FslUfnGetKitlDMABuffer     00022794 f   fsl_usbfn_rndiskitl_mx25_topaz_v1:stub.obj
 0001:000117ec       NANDBootReserved           000227ec f   nand_boot_common_topaz_v1:nandboot.obj
 0001:000118d4       GetNextGoodBlock           000228d4 f   nand_boot_common_topaz_v1:nandboot.obj
 0001:0001191c       GetPhyBlkAddr              0002291c f   nand_boot_common_topaz_v1:nandboot.obj
 0001:00011980       NANDWriteXldr              00022980 f   nand_boot_common_topaz_v1:nandboot.obj
 0001:00011ce8       NANDWriteBoot              00022ce8 f   nand_boot_common_topaz_v1:nandboot.obj
 0001:0001200c       NANDWriteNK                0002300c f   nand_boot_common_topaz_v1:nandboot.obj
 0001:000123a8       NANDLoadNK                 000233a8 f   nand_boot_common_topaz_v1:nandboot.obj
 0001:0001252c       NANDLoadBootCFG            0002352c f   nand_boot_common_topaz_v1:nandboot.obj
 0001:00012620       NANDStoreBootCFG           00023620 f   nand_boot_common_topaz_v1:nandboot.obj
 0001:00012784       NANDFormatNK               00023784 f   nand_boot_common_topaz_v1:nandboot.obj
 0001:000128ac       NANDWriteIPL               000238ac f   nand_boot_common_topaz_v1:nandboot.obj
 0001:00012bd4       IsSectorEmpty              00023bd4 f   nand_boot_common_topaz_v1:nandboot.obj
 0001:00012c38       NANDStartWriteBinDIO       00023c38 f   nand_boot_common_topaz_v1:nandboot.obj
 0001:00012dd0       NANDContinueWriteBinDIO    00023dd0 f   nand_boot_common_topaz_v1:nandboot.obj
 0001:00013060       NANDFinishWriteBinDIO      00024060 f   nand_boot_common_topaz_v1:nandboot.obj
 0001:000130a0       NANDLoadIPL                000240a0 f   nand_boot_common_topaz_v1:nandboot.obj
 0001:000131ec       NANDFormatAll              000241ec f   nand_boot_common_topaz_v1:nandboot.obj
 0001:000132ec       FMD_Init                   000242ec f   nand_common_topaz_v1:fmd.obj
 0001:0001348c       FMD_ReadSector             0002448c f   nand_common_topaz_v1:fmd.obj
 0001:000135cc       FMD_EraseBlock             000245cc f   nand_common_topaz_v1:fmd.obj
 0001:0001361c       FMD_WriteSector            0002461c f   nand_common_topaz_v1:fmd.obj
 0001:0001375c       FMD_GetInfo                0002475c f   nand_common_topaz_v1:fmd.obj
 0001:000137ec       FMD_GetBlockStatus         000247ec f   nand_common_topaz_v1:fmd.obj
 0001:0001389c       FMD_SetBlockStatus         0002489c f   nand_common_topaz_v1:fmd.obj
 0001:00013b44       ?BBT_GetBlockBadStatus@@YAHKK@Z 00024b44 f   nand_common_topaz_v1:bbt.obj
 0001:00013b98       ?BBT_SetBlockBadStatus@@YAXKK@Z 00024b98 f   nand_common_topaz_v1:bbt.obj
 0001:00014790       ?BBT_Init@@YAHXZ           00025790 f   nand_common_topaz_v1:bbt.obj
 0001:0001489c       BSPNAND_GetFlashInfo       0002589c f   nandfmd_lib:nandbsp.obj
 0001:00014970       BSPNAND_GetBufferPointer   00025970 f   nandfmd_lib:nandbsp.obj
 0001:000149b8       SDHCWriteXldr              000259b8 f   sdmmc_boot_common_topaz_v1:sdboot.obj
 0001:00014abc       SDHCWriteBoot              00025abc f   sdmmc_boot_common_topaz_v1:sdboot.obj
 0001:00014bb8       SDHCWriteNK                00025bb8 f   sdmmc_boot_common_topaz_v1:sdboot.obj
 0001:00014da4       SDHCLoadNK                 00025da4 f   sdmmc_boot_common_topaz_v1:sdboot.obj
 0001:00014eb0       SDHCFormatAll              00025eb0 f   sdmmc_boot_common_topaz_v1:sdboot.obj
 0001:00014fbc       SDHCCreateFileSystemPartition 00025fbc f   sdmmc_boot_common_topaz_v1:sdboot.obj
 0001:00015084       SDHCLoadBootCFG            00026084 f   sdmmc_boot_common_topaz_v1:sdboot.obj
 0001:0001516c       SDHCStoreBootCFG           0002616c f   sdmmc_boot_common_topaz_v1:sdboot.obj
 0001:00015264       EMMCToggleBP               00026264 f   sdmmc_boot_common_topaz_v1:sdboot.obj
 0001:000152ec       EMMCToggleBPSize           000262ec f   sdmmc_boot_common_topaz_v1:sdboot.obj
 0001:00015454       ESDSetActivePartition      00026454 f   sdmmc_boot_common_topaz_v1:sdboot.obj
 0001:00015518       ESDQueryPartitionSize      00026518 f   sdmmc_boot_common_topaz_v1:sdboot.obj
 0001:000155a8       ESDToggleBP                000265a8 f   sdmmc_boot_common_topaz_v1:sdboot.obj
 0001:000155ec       ESDToggleBPSize            000265ec f   sdmmc_boot_common_topaz_v1:sdboot.obj
 0001:00015700       SDHCDisableBP              00026700 f   sdmmc_boot_common_topaz_v1:sdboot.obj
 0001:00015748       SDCard_command_config      00026748 f   sdmmc_boot_common_topaz_v1:sdfmd.obj
 0001:00015764       SDMMC_GetInfo              00026764 f   sdmmc_boot_common_topaz_v1:sdfmd.obj
 0001:000157a4       SDMMC_get_cid              000267a4 f   sdmmc_boot_common_topaz_v1:sdfmd.obj
 0001:00015838       SDMMC_card_software_reset  00026838 f   sdmmc_boot_common_topaz_v1:sdfmd.obj
 0001:00015898       SDMMC_card_send_appcmd     00026898 f   sdmmc_boot_common_topaz_v1:sdfmd.obj
 0001:0001590c       SDMMC_get_csd              0002690c f   sdmmc_boot_common_topaz_v1:sdfmd.obj
 0001:000159ac       SDMMC_get_ext_csd          000269ac f   sdmmc_boot_common_topaz_v1:sdfmd.obj
 0001:00015a44       SDMMC_GetCardCapacity      00026a44 f   sdmmc_boot_common_topaz_v1:sdfmd.obj
 0001:00015b3c       SDMMC_set_blocklen         00026b3c f   sdmmc_boot_common_topaz_v1:sdfmd.obj
 0001:00015bac       SDMMC_send_rca             00026bac f   sdmmc_boot_common_topaz_v1:sdfmd.obj
 0001:00015c78       SDMMC_R1b_busy_wait        00026c78 f   sdmmc_boot_common_topaz_v1:sdfmd.obj
 0001:00015d48       SDMMC_EraseBlock           00026d48 f   sdmmc_boot_common_topaz_v1:sdfmd.obj
 0001:00015e78       SDMMC_ReadSector           00026e78 f   sdmmc_boot_common_topaz_v1:sdfmd.obj
 0001:00015f3c       SDMMC_WriteSector          00026f3c f   sdmmc_boot_common_topaz_v1:sdfmd.obj
 0001:00016014       SDMMC_Init                 00027014 f   sdmmc_boot_common_topaz_v1:sdfmd.obj
 0001:00016094       SDMMC_set_data_transfer_mode 00027094 f   sdmmc_boot_common_topaz_v1:sdfmd.obj
 0001:00016114       SD_VoltageValidation       00027114 f   sdmmc_boot_common_topaz_v1:sd.obj
 0001:00016364       SD_Init                    00027364 f   sdmmc_boot_common_topaz_v1:sd.obj
 0001:000164c8       MMC_Send_Switch_Cmd        000274c8 f   sdmmc_boot_common_topaz_v1:mmc.obj
 0001:00016538       MMC_Init                   00027538 f   sdmmc_boot_common_topaz_v1:mmc.obj
 0001:00016764       PrepareBuffer              00027764 f   oal_spifmd:cspifmd.obj
 0001:00016a90       SPIFMD_GetInfo             00027a90 f   oal_spifmd:cspifmd.obj
 0001:00016ad0       SPIFMD_GetBlockStatus      00027ad0 f   oal_spifmd:cspifmd.obj
 0001:00016ad8       SPIFMD_EraseBlock          00027ad8 f   oal_spifmd:cspifmd.obj
 0001:00016b28       SPIFMD_ReadSector          00027b28 f   oal_spifmd:cspifmd.obj
 0001:00016be0       SPIFMD_WriteSector         00027be0 f   oal_spifmd:cspifmd.obj
 0001:00016c90       SPIFMD_Init                00027c90 f   oal_spifmd:cspifmd.obj
 0001:00016e00       OALI2cEnable               00027e00 f   i2cutils:i2cutils.obj
 0001:00016e60       OALI2cDisable              00027e60 f   i2cutils:i2cutils.obj
 0001:00016e80       OALI2cCalculateClkRateDiv  00027e80 f   i2cutils:i2cutils.obj
 0001:00016f80       OALI2cGenerateStart        00027f80 f   i2cutils:i2cutils.obj
 0001:00017090       OALI2cRepeatedStart        00028090 f   i2cutils:i2cutils.obj
 0001:00017180       OALI2cGenerateStop         00028180 f   i2cutils:i2cutils.obj
 0001:00017260       OALI2cInit                 00028260 f   i2cutils:i2cutils.obj
 0001:0001733c       OALI2cWriteData            0002833c f   i2cutils:i2cutils.obj
 0001:00017490       OALI2cReadData             00028490 f   i2cutils:i2cutils.obj
 0001:0001767c       EbootInitTftpSimple        0002867c f   eboot:ebsimp.obj
 0001:000176e0       EbootEtherReadData         000286e0 f   eboot:ebsimp.obj
 0001:0001786c       EbootCheckIP               0002886c f   eboot:ebsimp.obj
 0001:0001793c       EbootGetDHCPAddr           0002893c f   eboot:ebsimp.obj
 0001:00017b08       EbootSendBootmeAndWaitForTftp 00028b08 f   eboot:ebsimp.obj
 0001:00017cd4       EbootWaitForHostConnect    00028cd4 f   eboot:ebsimp.obj
 0001:00017e58       EbootInitEtherTransport    00028e58 f   eboot:ebsimp.obj
 0001:00017f54       EbootInitTFtpd             00028f54 f   eboot:tftpd.obj
 0001:00017f74       tolower                    00028f74 f   eboot:tftpd.obj
 0001:00017f84       EbootTFtpdServerRegister   00028f84 f   eboot:tftpd.obj
 0001:00018010       GenerateSrcPort            00029010 f   eboot:tftpd.obj
 0001:0001801c       TFtpdCallBack              0002901c f   eboot:tftpd.obj
 0001:000182fc       TFtpdFormNewLink           000292fc f   eboot:tftpd.obj
 0001:00018710       EbootInitTFtp              00029710 f   eboot:tftp.obj
 0001:00018760       TFtpKillLink               00029760 f   eboot:tftp.obj
 0001:00018858       TFtpStateMachine           00029858 f   eboot:tftp.obj
 0001:00018af8       EbootTFtpReceiver          00029af8 f   eboot:tftp.obj
 0001:00018c60       SrcAddrFromFrame           00029c60 f   eboot:udp.obj
 0001:00018cc8       EbootGratuitousARP         00029cc8 f   eboot:udp.obj
 0001:00018e1c       SetPromiscuousIP           00029e1c f   eboot:udp.obj
 0001:00018e30       ClearPromiscuousIP         00029e30 f   eboot:udp.obj
 0001:00018ef8       EbootProcessARP            00029ef8 f   eboot:udp.obj
 0001:00019188       EbootSendUDP               0002a188 f   eboot:udp.obj
 0001:00019410       EbootCheckUDP              0002a410 f   eboot:udp.obj
 0001:000196e0       DHCPBuildOps               0002a6e0 f   eboot:dhcp.obj
 0001:00019894       DHCPFindOption             0002a894 f   eboot:dhcp.obj
 0001:00019988       EbootProcessDHCP           0002a988 f   eboot:dhcp.obj
 0001:00019cd0       EbootInitDHCP              0002acd0 f   eboot:dhcp.obj
 0001:00019d34       EbootDHCPRetransmit        0002ad34 f   eboot:dhcp.obj
 0001:00019e58       SendDHCP                   0002ae58 f   eboot:dhcp.obj
 0001:0001a2e4       EbootDHCPDecline           0002b2e4 f   eboot:dhcp.obj
 0001:0001a360       EbootProcessEDBG           0002b360 f   eboot:edbg.obj
 0001:0001a528       EbootSendBootme            0002b528 f   eboot:edbg.obj
 0001:0001a700       __report_gsfailure         0002b700 f   gsnull:gsnull.obj
 0001:0001a704       __GSHandlerCheckCommon     0002b704 f   fulllibc:gshandler.obj
 0001:0001a73c       __GSHandlerCheck           0002b73c f   fulllibc:gshandler.obj
 0001:0001a75c       __security_check_cookie    0002b75c f   fulllibc:armsecgs.obj
 0001:0001a76c       __gsfailure                0002b76c     fulllibc:armsecgs.obj
 0001:0001a7b0       atoi                       0002b7b0 f   fulllibc:atox.obj
 0001:0001a7bc       __rt_udivrem64by64         0002b7bc     fulllibc:mdsdiv64.obj
 0001:0001a8b4       __rt_divrem64by64          0002b8b4     fulllibc:mdsdiv64.obj
 0001:0001a904       __rt_udiv64by64            0002b904     fulllibc:mdsdiv64.obj
 0001:0001a914       __rt_urem64by64            0002b914     fulllibc:mdsdiv64.obj
 0001:0001a92c       __rt_sdiv64by64            0002b92c     fulllibc:mdsdiv64.obj
 0001:0001a93c       __rt_srem64by64            0002b93c     fulllibc:mdsdiv64.obj
 0001:0001a954       __rt_udiv                  0002b954 f   fulllibc:__udiv.obj
 0001:0001aa18       strncmp                    0002ba18     fulllibc:astrncmp.obj
 0001:0001aa48       memset                     0002ba48     fulllibc:memset.obj
 0001:0001aad0       memcmp                     0002bad0     fulllibc:memcmp.obj
 0001:0001aba0       memcpy                     0002bba0 f   fulllibc:memcpy.obj
 0001:0001b540       strlen                     0002c540     fulllibc:mdsstrlen.obj
 0001:0001b5a4       strncpy_s                  0002c5a4 f   fulllibc:strncpy_s.obj
 0001:0001b6cc       memmove                    0002c6cc     fulllibc:memmove.obj
 0001:0001be5c       memmovebigblk              0002ce5c     fulllibc:memmove.obj
 0001:0001c8f4       __rt_sdiv                  0002d8f4 f   fulllibc:__div.obj
 0001:0001c9d0       strcat                     0002d9d0     fulllibc:mdsstrcat.obj
 0001:0001c9f8       strcpy_s                   0002d9f8 f   fulllibc:strcpy_s.obj
 0001:0001ca9c       strcmp                     0002da9c     fulllibc:mdsstrcmp.obj
 0001:0001ccb4       _itoa_s                    0002dcb4 f   fulllibc:xtoas.obj
 0001:0001ccf8       strcat_s                   0002dcf8 f   fulllibc:strcat_s.obj
 0001:0001d008       strtol                     0002e008 f   fulllibc:strtol.obj
 0001:0001d010       __raise_int_divide_by_zero 0002e010 f   fulllibc:diverr.obj
 0001:0001d028       _invalid_parameter         0002e028 f   fulllibc:invarg.obj
 0001:0001d094       __crtRaiseException        0002e094 f   fulllibc:raiseexc.obj
 0001:0001d0b8       _decode_pointer            0002e0b8 f   fulllibc:encptr.obj
 0001:0001d0bc       OALFlushDCache             0002e0bc f   oal_cache_arm926:flushdc.obj
 0001:0001d0c8       OALCleanDCache             0002e0c8 f   oal_cache_arm926:cleandc.obj
 0001:0001d0d4       OALFlushDCacheLines        0002e0d4 f   oal_cache_arm926:flushdclines.obj
 0001:0001d0f4       NKDbgPrintfW               0002e0f4 f   oal_blnk:wrappers.obj
 0001:0001d128       NKwvsprintfW               0002e128 f   oal_blnk:format.obj
 0001:0001e518       BootloaderMain             0002f518 f   oal_blcommon:blcommon.obj
 0001:0001e77c       OALLogSetZones             0002f77c f   oal_log:debug.obj
 0001:0001e78c       OALKitlCreateName          0002f78c f   oal_kitl:name.obj
 0001:0001e878       OALKitlIPtoString          0002f878 f   oal_kitl:format.obj
 0001:0001e8cc       OALKitlMACtoString         0002f8cc f   oal_kitl:format.obj
 0001:0001e930       OALKitlStringToIP          0002f930 f   oal_kitl:format.obj
 0001:0001e9bc       OALKitlStringToMAC         0002f9bc f   oal_kitl:format.obj
 0001:0001eafc       OEMWriteDebugString        0002fafc f   oal_other:debug.obj
 0001:0001eb24       BSP_GetNANDBufferPointer   0002fb24 f   bootcmn:nand.obj
 0001:0001eb3c       BSP_GetNANDImageCfg        0002fb3c f   bootcmn:nand.obj
 0001:0001eb94       SDConfigPins               0002fb94 f   bootcmn:esdhc.obj
 0001:0001ec88       SDHC_IsCardWriteProtected  0002fc88 f   bootcmn:esdhc.obj
 0001:0001eca8       SetClockRate               0002fca8 f   bootcmn:esdhc.obj
 0001:0001efdc       SDHCSendCmdWaitResp        0002ffdc f   bootcmn:esdhc.obj
 0001:0001f01c       SDHCReadResponse           0003001c f   bootcmn:esdhc.obj
 0001:0001f0dc       SDHCDataRead               000300dc f   bootcmn:esdhc.obj
 0001:0001f170       SDHCDataWrite              00030170 f   bootcmn:esdhc.obj
 0001:0001f208       BSP_MMC4BitSupported       00030208 f   bootcmn:esdhc.obj
 0001:0001f210       BSP_GetSDImageCfg          00030210 f   bootcmn:esdhc.obj
 0001:0001f25c       SDInterface_Init           0003025c f   bootcmn:esdhc.obj
 0001:0001f34c       OutputHelpInformation      0003034c f   bootshell_common_topaz_v1:bootshell.obj
 0001:0001f3b4       HexString2Hex              000303b4 f   bootshell_common_topaz_v1:bootshell.obj
 0001:0001f5d4       SetReg                     000305d4 f   bootshell_common_topaz_v1:bootshell.obj
 0001:0001f640       ShowReg                    00030640 f   bootshell_common_topaz_v1:bootshell.obj
 0001:0001f69c       SetBit                     0003069c f   bootshell_common_topaz_v1:bootshell.obj
 0001:0001f758       DebugGetLine               00030758 f   bootshell_common_topaz_v1:bootshell.obj
 0001:0001f7d8       ?SwapBBI@@YAXXZ            000307d8 f   nand_mx25_topaz_v1:cspnand.obj
 0001:0001f8d0       ?NFCAlloc@@YAHXZ           000308d0 f   nand_mx25_topaz_v1:cspnand.obj
 0001:0001f900       ?NFCSetPagesize@@YAHI@Z    00030900 f   nand_mx25_topaz_v1:cspnand.obj
 0001:0001f980       ?NFCWait@@YAXXZ            00030980 f   nand_mx25_topaz_v1:cspnand.obj
 0001:0001f9c4       CSPNAND_Reset              000309c4 f   nand_mx25_topaz_v1:cspnand.obj
 0001:0001f9fc       CSPNAND_ReadID             000309fc f   nand_mx25_topaz_v1:cspnand.obj
 0001:0001fa74       CSPNAND_EnableECC          00030a74 f   nand_mx25_topaz_v1:cspnand.obj
 0001:0001fab8       CSPNAND_ILSupport          00030ab8 f   nand_mx25_topaz_v1:cspnand.obj
 0001:0001fac0       CSPNAND_PostInit           00030ac0 f   nand_mx25_topaz_v1:cspnand.obj
 0001:0001fac4       CSPNAND_Init               00030ac4 f   nand_mx25_topaz_v1:cspnand.obj
 0001:0001fc10       CSPNAND_ReadSector         00030c10 f   nand_mx25_topaz_v1:cspnand.obj
 0001:0001ffb0       CSPNAND_EraseBlock         00030fb0 f   nand_mx25_topaz_v1:cspnand.obj
 0001:000200f0       CSPNAND_WriteSector        000310f0 f   nand_mx25_topaz_v1:cspnand.obj
 0001:000203d8       CSPNAND_GetECCStatus       000313d8 f   nand_mx25_topaz_v1:cspnand.obj
 0001:00020418       RdPageAlign4               00031418 f   nand_mx25_topaz_v1:nfcrw.obj
 0001:0002043c       RdPageAlign1               0003143c f   nand_mx25_topaz_v1:nfcrw.obj
 0001:000204ac       RdPageAlign2               000314ac f   nand_mx25_topaz_v1:nfcrw.obj
 0001:00020514       RdPageAlign3               00031514 f   nand_mx25_topaz_v1:nfcrw.obj
 0001:00020584       WrPageAlign4               00031584 f   nand_mx25_topaz_v1:nfcrw.obj
 0001:000205a8       WrPageAlign1               000315a8 f   nand_mx25_topaz_v1:nfcrw.obj
 0001:00020618       WrPageAlign2               00031618 f   nand_mx25_topaz_v1:nfcrw.obj
 0001:00020680       WrPageAlign3               00031680 f   nand_mx25_topaz_v1:nfcrw.obj
 0001:000206f4       __crt_unrecoverable_error  000316f4 f   eboot:crtsupp.obj
 0001:000206f8       OALLogPrintf               000316f8 f   oal_log:log.obj
 0001:00020720       BSPNAND_RemapRegister      00031720 f   bootcmn:nfc_boot.obj
 0002:00000000       EthDevice                  00032000     eboot.obj
 0002:00000270       g_DownloadImage            00032270     bootcmn:main.obj
 0002:00000350       Am79c874Info               00032350     oal_ethdrv_fec_common_topaz_v1:fec.obj
 0002:00000554       PhyInfo                    00032554     oal_ethdrv_fec_common_topaz_v1:fec.obj
 0002:00000568       LAN8700Info                00032568     oal_ethdrv_fec_common_topaz_v1:fec.obj
 0002:00000770       Dp83640Info                00032770     oal_ethdrv_fec_common_topaz_v1:fec.obj
 0002:00000978       KSZ8041NLInfo              00032978     oal_ethdrv_fec_common_topaz_v1:fec.obj
 0002:00000b7c       bRndisSendPacketEmpty      00032b7c     fsl_rne_mdd_common_topaz_v1:rndis.obj
 0002:00000bb0       RNdisMddSupportedOids      00032bb0     fsl_rne_mdd_common_topaz_v1:hostmini.obj
 0002:00000c40       g_InterruptData            00032c40     fsl_rne_pdd_common_topaz_v1:rndis_pdd.obj
 0002:00001000       g_serial_rev_buf           00033000     fsl_rne_pdd_common_topaz_v1:buffer.obj
 0002:00001000       g_rndis_ep2_buf            00033000     fsl_rne_pdd_common_topaz_v1:buffer.obj
 0002:00003000       g_serial_send_buf          00035000     fsl_rne_pdd_common_topaz_v1:buffer.obj
 0002:00003000       g_rndis_ep3_buf            00035000     fsl_rne_pdd_common_topaz_v1:buffer.obj
 0002:00005000       g_rndis_ep0_buf            00037000     fsl_rne_pdd_common_topaz_v1:buffer.obj
 0002:00005440       ?ChipInfo@@3PAU_NandChipInfo@@A 00037440     nand_common_topaz_v1:fmd.obj
 0002:00005570       __security_cookie          00037570     gsnull:gsnull.obj
 0002:00005574       __security_cookie_complement 00037574     gsnull:gsnull.obj
 0002:000055c0       initialOALLogZones         000375c0     oal_log:debug.obj
 0002:000055c8       dpCurSettings              000375c8     oal_log:debug.obj
 0002:00005bb0       g_bNandBootloader          00037bb0     bootcmn:main.obj
 0002:00005bb4       g_bNandExist               00037bb4     bootcmn:main.obj
 0002:00005bb8       g_bSDHCBootloader          00037bb8     bootcmn:main.obj
 0002:00005bbc       g_bSDHCExist               00037bbc     bootcmn:main.obj
 0002:00005bc0       g_bSpiBootloader           00037bc0     bootcmn:main.obj
 0002:00005bc4       g_bSpiExist                00037bc4     bootcmn:main.obj
 0002:00005bc8       g_SerialUSBDownload        00037bc8     bootcmn:main.obj
 0002:00005c08       bCFGChanged                00037c08     blmenu_common_topaz_v1:menu.obj
 0002:00005c0c       PrintSoc                   00037c0c     blmenu_common_topaz_v1:menu.obj
 0002:0000fb40       g_pEP3DataWrapper          00041b40     fsl_rne_pdd_common_topaz_v1:rndis_pdd.obj
 0002:0000fb44       g_devState                 00041b44     fsl_rne_pdd_common_topaz_v1:rndis_pdd.obj
 0002:0000fb48       g_EP0TransferState         00041b48     fsl_rne_pdd_common_topaz_v1:rndis_pdd.obj
 0002:0000fb4c       g_EP2TransferState         00041b4c     fsl_rne_pdd_common_topaz_v1:rndis_pdd.obj
 0002:00010ea8       ?g_buffer@@3PAEA           00042ea8     oal_blserial:serfuncs.obj
 0002:00011ac0       ?g_mddInterface@@3U_UFN_MDD_INTERFACE_INFO@@A 00043ac0     fsl_serial_pdd_common_topaz_v1:serial_dl.obj
 0002:00011ac8       ?g_EP1Transfer@@3U_STransfer@@A 00043ac8     fsl_serial_pdd_common_topaz_v1:serial_dl.obj
 0002:00011ae8       ?g_RecvBuffer@@3PAEA       00043ae8     fsl_serial_pdd_common_topaz_v1:serial_dl.obj
 0002:00011b08       ?g_pddInterface@@3U_UFN_PDD_INTERFACE_INFO@@A 00043b08     fsl_serial_pdd_common_topaz_v1:serial_dl.obj
 0002:00011b68       ?g_EP2Transfer@@3U_STransfer@@A 00043b68     fsl_serial_pdd_common_topaz_v1:serial_dl.obj
 0002:00011b88       ?g_EP0Transfer@@3U_STransfer@@A 00043b88     fsl_serial_pdd_common_topaz_v1:serial_dl.obj
 0002:00011bec       ?g_DeviceState@@3W4DEVICE_STATE@@A 00043bec     fsl_serial_pdd_common_topaz_v1:serial_dl.obj
 0002:00011bf0       ?g_EP0State@@3W4TRANSFER_STATE@@A 00043bf0     fsl_serial_pdd_common_topaz_v1:serial_dl.obj
 0002:00011bf4       ?g_EP1State@@3W4TRANSFER_STATE@@A 00043bf4     fsl_serial_pdd_common_topaz_v1:serial_dl.obj
 0002:00011bf8       ?g_EP2State@@3W4TRANSFER_STATE@@A 00043bf8     fsl_serial_pdd_common_topaz_v1:serial_dl.obj
 0002:00011bfc       ?g_RecvBufferHead@@3GA     00043bfc     fsl_serial_pdd_common_topaz_v1:serial_dl.obj
 0002:00011c00       ?g_RecvBufferTail@@3GA     00043c00     fsl_serial_pdd_common_topaz_v1:serial_dl.obj
 0002:00011c64       ?g_FlashInfoExt@@3U_FlashInfoExt@@A 00043c64     nand_common_topaz_v1:fmd.obj
 0002:00011c9c       ?g_bInterLeaveMode@@3HA    00043c9c     nand_common_topaz_v1:fmd.obj
 0002:00011cc8       ?g_SectorBuf@@3PAEA        00043cc8     nandfmd_lib:nandbsp.obj
 0002:000124c8       ?g_BBTSecondBuf@@3PAEA     000444c8     nandfmd_lib:nandbsp.obj
 0002:00012cc8       ?g_BBTFirstBuf@@3PAEA      00044cc8     nandfmd_lib:nandbsp.obj
 0002:000134c8       ?BBMarkPage@@3PAEA         000454c8     nandfmd_lib:nandbsp.obj
 0002:000134d0       eSDBPEnabled               000454d0     sdmmc_boot_common_topaz_v1:sdboot.obj
 0002:000134d8       bCacheBuffer               000454d8     sdmmc_boot_common_topaz_v1:sdboot.obj
 0002:000136d8       Card_rca                   000456d8     sdmmc_boot_common_topaz_v1:sdfmd.obj
 0002:000136dc       bHighDensityCard           000456dc     sdmmc_boot_common_topaz_v1:sdfmd.obj
 0002:000136e0       mmcSpecVersion             000456e0     sdmmc_boot_common_topaz_v1:sdfmd.obj
 0002:000136e4       eSDBootPartitionSize       000456e4     sdmmc_boot_common_topaz_v1:sd.obj
 0002:0001fdf0       bDoLaunch                  00051df0     eboot:tftpd.obj
 0002:0001fdf4       TftpPeerAddr               00051df4     eboot:tftpd.obj
 0002:00021e28       bLastCmdRead               00053e28     bootcmn:esdhc.obj
 0002:00021e2c       ?bECCMode@@3_NA            00053e2c     nand_mx25_topaz_v1:cspnand.obj
 0002:00021e30       ?g_CSPfi@@3U_FlashInfoExt@@A 00053e30     nand_mx25_topaz_v1:cspnand.obj
 0002:00021e68       g_pNFC                     00053e68     nand_mx25_topaz_v1:cspnand.obj
 0002:00021e70       g_DeviceAddr               00053e70     <common>
 0002:00021e80       g_oalCacheInfo             00053e80     <common>
 0002:00021ec8       g_pOEMVerifyMemory         00053ec8     <common>
 0002:00021ecc       g_dwROMOffset              00053ecc     <common>
 0002:00021ed0       g_pOEMReportError          00053ed0     <common>
 0002:00021ed4       g_pOEMMultiBINNotify       00053ed4     <common>
 0002:00021ed8       g_pOEMCheckSignature       00053ed8     <common>
 0002:00021edc       g_pDdkClkConfig            00053edc     <common>
 0002:00021ee0       g_pUART                    00053ee0     <common>
 0002:00021ee4       g_pIOMUX                   00053ee4     <common>
 0002:00021ee8       g_pCRM                     00053ee8     <common>
 0002:00021eec       dwVVN                      00053eec     <common>
 0002:00021ef0       g_pESDHCReg                00053ef0     <common>
 0002:00021ef4       g_pGPIO4                   00053ef4     <common>
 0002:00021f00       sectorBuf                  00053f00     <common>
 0002:00022f00       pfnEDbgDisableInts         00054f00     <common>
 0002:00022f04       pfnEDbgGetFrame            00054f04     <common>
 0002:00022f08       pfnEDbgEnableInts          00054f08     <common>
 0002:00022f0c       pfnEDbgInit                00054f0c     <common>
 0002:00022f10       pfnEDbgSendFrame           00054f10     <common>
 0002:00022f14       pfnEDbgInitDMABuffer       00054f14     <common>
 0002:00022f18       g_pBSPArgs                 00054f18     <common>
 0002:00022f1c       g_ImageType                00054f1c     <common>
 0002:00022f20       g_ImageMemory              00054f20     <common>
 0002:00022f24       g_DefaultRamAddress        00054f24     <common>
 0002:00022f30       g_BinDIO                   00054f30     <common>
 0002:00022f40       g_BootCFG                  00054f40     <common>
 0002:00022f9c       SetBitFlag                 00054f9c     <common>
 0002:00022fa0       SetRegFlag                 00054fa0     <common>
 0002:00022fa4       ExitingShellFlag           00054fa4     <common>
 0002:00022fa8       ShowRegFlag                00054fa8     <common>
 0002:00022fb0       BspValueSet                00054fb0     <common>
 0002:00022fba       BspBitSet                  00054fba     <common>
 0002:00022fc0       Linebuffer                 00054fc0     <common>
 0002:000231c0       BspAddrSet                 000551c0     <common>
 0002:000231e0       RndisMdd                   000551e0     <common>
 0002:000232b0       g_EP0DataWrapper           000552b0     <common>
 0002:000232c0       MDDZONE5                   000552c0     <common>
 0002:000232c8       g_mddInterface             000552c8     <common>
 0002:000232e0       g_EP1Transfer              000552e0     <common>
 0002:00023300       g_RndisKitlDev             00055300     <common>
 0002:00023748       g_udr                      00055748     <common>
 0002:00023750       MDDZONE4                   00055750     <common>
 0002:00023754       PDDZONE                    00055754     <common>
 0002:00023760       g_EP3Transfer              00055760     <common>
 0002:00023780       g_pddInterface             00055780     <common>
 0002:000237e0       MDDZONE3                   000557e0     <common>
 0002:00023800       g_EP2Transfer              00055800     <common>
 0002:00023820       PDDZONE0                   00055820     <common>
 0002:00023840       g_EP0Transfer              00055840     <common>
 0002:00023860       MDDZONE0                   00055860     <common>
 0002:00023864       MDDZONE                    00055864     <common>
 0002:00023868       MDDZONE2                   00055868     <common>
 0002:00023880       g_csRegister               00055880     <common>
 0002:000238a0       extCSDBuffer               000558a0     <common>
 0002:00023aa0       sdCardReg                  00055aa0     <common>
 0002:00023ae0       SDImageCfg                 00055ae0     <common>
 0002:00023b20       SDController               00055b20     <common>
 0002:00023bc8       g_pCspi                    00055bc8     <common>
 0002:00023be0       TFtpLinks                  00055be0     <common>
 0002:000244a0       wOdoWellKnownServerPort    000564a0     <common>
 0002:000244a2       wHostWellKnownServerPort   000564a2     <common>
 0002:000244a4       nNumTFtpLinksInUse         000564a4     <common>
 0002:000244c0       TFTPFrameBuffer            000564c0     <common>
 0002:00024900       TFtpdServerRegistry        00056900     <common>
 0002:000249c8       __pInvalidArgHandler       000569c8     <common>

 entry point at        0001:00000000

 Static symbols

 0001:0000584c       SelectEtherDevice          0001684c f   menu.obj
 0001:00005894       SelectSerialDebug          00016894 f   menu.obj
 0001:000058ec       SelectBootDevice           000168ec f   menu.obj
 0001:00005934       PrintData                  00016934 f   menu.obj
 0001:00007b1c       InitUSBRNDISDevice         00018b1c f   bootcmn:ether.obj
 0001:00009d98       ParseCommand               0001ad98 f   bsp_bootshell:bspbootshell.obj
 0001:0000c160       PDD_SendNotification       0001d160 f   fsl_rne_pdd_common_topaz_v1:rndis_pdd.obj
 0001:0000c188       PDD_RecvNotification       0001d188 f   fsl_rne_pdd_common_topaz_v1:rndis_pdd.obj
 0001:0000c694       RegisterUSBDevice          0001d694 f   fsl_rne_pdd_common_topaz_v1:rndis_pdd.obj
 0001:0000d204       CeLogMsg                   0001e204 f   usb_usbfn_mx25_topaz_v1:i_pdd.obj
 0001:0000d2dc       GetSetupPacket             0001e2dc f   usb_usbfn_mx25_topaz_v1:i_pdd.obj
 0001:0000d3a4       InitQh0                    0001e3a4 f   usb_usbfn_mx25_topaz_v1:i_pdd.obj
 0001:0000d67c       PrimeQh0ForZeroTransfer    0001e67c f   usb_usbfn_mx25_topaz_v1:i_pdd.obj
 0001:0000d8bc       HandleUSBReset             0001e8bc f   usb_usbfn_mx25_topaz_v1:i_pdd.obj
 0001:0000dee0       BuildTdBufferList          0001eee0 f   usb_usbfn_mx25_topaz_v1:i_pdd.obj
 0001:00010b20       ?HandleUSBDeviceRegistration@@YAXXZ 00021b20 f   fsl_serial_pdd_common_topaz_v1:serial_dl.obj
 0001:00010f64       ?HandleSetupPkt@@YAXPAU_USB_DEVICE_REQUEST@@PAU_EP0_REQUEST@@@Z 00021f64 f   fsl_serial_pdd_common_topaz_v1:serial_dl.obj
 0001:00011090       ?HandlePDDNotification@@YAHPAXKK@Z 00022090 f   fsl_serial_pdd_common_topaz_v1:serial_dl.obj
 0001:000117a0       NANDBootInit               000227a0 f   nand_boot_common_topaz_v1:nandboot.obj
 0001:000139a4       ?ReadBlockBadStatus@@YAHKK@Z 000249a4 f   nand_common_topaz_v1:bbt.obj
 0001:00013ae4       ?BBT_GetSectorAddr@@YAKK@Z 00024ae4 f   nand_common_topaz_v1:bbt.obj
 0001:00013bf4       ?BBT_EraseOperation@@YAHKK@Z 00024bf4 f   nand_common_topaz_v1:bbt.obj
 0001:00013c58       ?ReadBBTSignature@@YAHKK@Z 00024c58 f   nand_common_topaz_v1:bbt.obj
 0001:00013d04       ?WriteBBTSignature@@YAHKK@Z 00024d04 f   nand_common_topaz_v1:bbt.obj
 0001:00013d94       ?WriteBBT@@YAHKK@Z         00024d94 f   nand_common_topaz_v1:bbt.obj
 0001:00014014       ?ReadBBT@@YAHXZ            00025014 f   nand_common_topaz_v1:bbt.obj
 0001:00014664       ?CreateBBT@@YAHXZ          00025664 f   nand_common_topaz_v1:bbt.obj
 0001:00016264       SDGetBitMode               00027264 f   sdmmc_boot_common_topaz_v1:sd.obj
 0001:00016818       TransactMessage            00027818 f   oal_spifmd:cspifmd.obj
 0001:000169d0       FlashIsWriteable           000279d0 f   oal_spifmd:cspifmd.obj
 0001:00016a40       WriteEnable                00027a40 f   oal_spifmd:cspifmd.obj
 0001:000175fc       EbootSimpleCallback        000285fc f   eboot:ebsimp.obj
 0001:00018e44       CRC                        00029e44 f   eboot:udp.obj
 0001:00019624       FormatDHCPName             0002a624 f   eboot:dhcp.obj
 0001:0001cb8c       xtoa_s                     0002db8c f   fulllibc:xtoas.obj
 0001:0001cde4       strtoxl                    0002dde4 f   fulllibc:strtol.obj
 0001:0001da4c       DownloadNB0                0002ea4c f   oal_blcommon:blcommon.obj
 0001:0001dc30       WriteImageToFlash          0002ec30 f   oal_blcommon:blcommon.obj
 0001:0001dd08       IsKernelRegion             0002ed08 f   oal_blcommon:blcommon.obj
 0001:0001ddbc       DownloadBin                0002edbc f   oal_blcommon:blcommon.obj
 0001:0001e1d4       DownloadImage              0002f1d4 f   oal_blcommon:blcommon.obj
 0001:0001ee04       SDHCCmdConfig              0002fe04 f   bootcmn:esdhc.obj
 0001:0001f878       ?SetCs@@YAXK@Z             00030878 f   nand_mx25_topaz_v1:cspnand.obj
